:0200000480007A
:10000000B72F0000938F0F8073900F306F00400365
:100010001300000013000000130000001300000094
:100020001300000013000000130000001300000084
:100030001300000013000000130000001300000074
:100040009702000093824211739052309300000097
:10005000130100009301000013020000930200004E
:100060001303000093030000130400009304000036
:10007000130500009305000013060000930600001E
:100080001307000093070000130800009308000006
:100090001309000093090000130A0000930A0000EE
:1000A000130B0000930B0000130C0000930C0000D6
:1000B000130D0000930D0000130E0000930E0000BE
:1000C000130F0000930F000097110200938141C1AC
:1000D0001705020013050543979503009385856A6C
:1000E00013060000EF00001A17050200130545383B
:1000F000970502009385653E13060000EF00801807
:1001000017A503001305456897B503009385856718
:1001100037B6ABAB1306B6BAEF00C01617B1030083
:1001200013018166EF70D07F9392120093D2120078
:100130009382D2FF638A02008322010013014100EF
:100140006F0000177300203083220100130141006B
:10015000730020301301C1FF23205100F32220340B
:10016000E3C402FC8322010013014100130141F8A2
:1001700023221100232421002326310023284100BB
:10018000232A5100232C6100232E71002320810299
:10019000232291022324A1022326B1022328C10293
:1001A000232AD102232CE102232EF1022320010570
:1001B0002322110523242105232631052328410567
:1001C000232A5105232C6105232E71052320810745
:1001D000232291072324A1072326B1072328C1073F
:1001E000232AD107232CE107232EF107732520347E
:1001F000F3251034130601006F000000731015344E
:1002000083204100032181008321C10003220101D9
:1002100083224101032381018323C10103240102BD
:1002200083244102032581028325C10203260103A1
:1002300083264103032781038327C1030328010485
:1002400083284104032981048329C104032A010569
:10025000832A4105032B8105832BC105032C01064D
:10026000832C4106032D8106832DC106032E010731
:10027000832E4107032F8107832FC1071301C10775
:10028000730020302320C5006376B50013054500B8
:100290006FF05FFF678000000000000000000000BA
:1002A000000000000000000000000000000000004E
:1002B000130101F8232011002322210023243100FF
:1002C0002326410023285100232A6100232C71009A
:1002D000232E8100232091022322A1022324B10294
:1002E0002326C1022328D102232AE102232CF10272
:1002F000232E010323201105232221052324310568
:100300002326410523285105232A6105232C710545
:10031000232E8105232091072322A1072324B1073F
:100320002326C1072328D107232AE107232CF1071D
:100330009702020083A2021723A02200F3221034A6
:10034000232E5106EF00C03B170102000321811547
:10035000032101008322C10773901234B7220000E9
:100360009382028873A00230832001000322C1001F
:100370008322010103234101832381010324C1015D
:100380008324010203254102832581020326C10241
:100390008326010303274103832781030328C10325
:1003A000832801040329410483298104032AC10409
:1003B000832A0105032B4105832B8105032CC105ED
:1003C000832C0106032D4106832D8106032EC106D1
:1003D000832E0107032F4107832F81071301010893
:1003E00073002030970202009382C21123A01200F2
:1003F00023A2220023A4320023A6420023A85200F5
:1004000023AA620023AC720023AE820023A09202D2
:1004100023A2A20223A4B20223A6C20223A8D202CC
:1004200023AAE20223ACF20223AE020323A01205A8
:1004300023A2220523A4320523A6420523A85205A0
:1004400023AA620523AC720523AE820523A092077E
:1004500023A2A20723A4B20723A6C20723A8D20778
:1004600023AAE20723ACF207EF60D02617010200AF
:1004700003214103032101008322C1077390123439
:10048000B72200009382028873A00230832001000B
:100490000322C1008322010103234101832381013F
:1004A0000324C10183240102032541028325810223
:1004B0000326C10283260103032741038327810307
:1004C0000328C103832801040329410483298104EB
:1004D000032AC104832A0105032B4105832B8105CF
:1004E000032CC105832C0106032D4106832D8106B3
:1004F000032EC106832E0107032F4107832F810797
:10050000130101087300203097020200938282FFDA
:1005100083A0020003A1420083A1820003A2C200C3
:1005200083A2020103A3420183A3820103A4C201A7
:1005300083A4020203A5420283A5820203A6C2028B
:1005400083A6020303A7420383A7820303A8C2036F
:1005500083A8020403A9420483A9820403AAC20453
:1005600083AA020503AB420583AB820503ACC20537
:1005700083AC020603AD420683AD820603AEC2061B
:1005800083AE020703AFC20983AF82076780000012
:1005900073700430130101F823201100232221007D
:1005A000232431002326410023285100232A6100FF
:1005B000232C7100232E8100232091022322A102EB
:1005C0002324B1022326C1022328D102232AE102D7
:1005D000232CF102232E01032320110523222105C0
:1005E000232431052326410523285105232A6105AB
:1005F000232C7105232E8105232091072322A10797
:100600002324B1072326C1072328D107232AE10782
:10061000232CF1079702020083A2C2E823A0220044
:10062000232E1106EF30402817010200032181E735
:10063000032101008322C10773901234B722000006
:100640009382028873A00230832001000322C1003C
:100650008322010103234101832381010324C1017A
:100660008324010203254102832581020326C1025E
:100670008326010303274103832781030328C10342
:10068000832801040329410483298104032AC10426
:10069000832A0105032B4105832B8105032CC1050A
:1006A000832C0106032D4106832D8106032EC106EE
:1006B000832E0107032F4107832F810713010108B0
:1006C00073002030737004306F00000073104530E9
:1006D000678000007325403073F04330678000006E
:1006E00097070000938747FE232EB5FE2322C5FA05
:1006F000232635F82320F5F8130505F86780000058
:10070000130101FF23261100EF608079EF20805054
:10071000631805008320C1001301010167800000F8
:100720008320C100130101016F3000189307850079
:100730001307F0FF2322F5002324E5002326F5000C
:100740002328F500232005006780000023280500EA
:10075000678000008327450023A2F50003A78700D8
:1007600023A4E50003A787002322B70023A4B70032
:1007700023A8A50083270500938717002320F500F1
:100780006780000003A605009307F0FF13078500AC
:100790006316F6006F008003138707008327470066
:1007A00083A60700E37AD6FE23A2F50023A4B700B0
:1007B00023A4E5002322B70023A8A5008327050072
:1007C000938717002320F5006780000003270501A9
:1007D000832747006FF05FFD0327450083268500D0
:1007E000832705012324D70003278500832645009E
:1007F0002322D70003A747006316A700032785001D
:1008000023A2E7002328050003A507001305F5FF31
:1008100023A0A70067800000032605049387050036
:10082000630406028325C50003274500B385C50080
:100830002326B50063E6E500832505002326B500E1
:10084000138507006F50004267800000130101FF0D
:100850002324810023261100130405002322910084
:10086000EF30D03783278404635AF004832744028F
:1008700063860704930444026F0000028327840404
:100880009387F7FF2324F404832784046358F0023A
:10089000832744026384070213850400EF3000635A
:1008A000E30E05FCEF30D00F832784049387F7FF16
:1008B0002324F40483278404E34CF0FC9307F0FF23
:1008C0002324F404EF30D034EF3050318327440434
:1008D000635AF00483270401638607049304040128
:1008E0006F000002832744049387F7FF2322F40458
:1008F000832744046358F0028327040163840702BA
:1009000013850400EF30805CE30E05FCEF305009E6
:10091000832744049387F7FF2322F40483274404A6
:10092000E34CF0FC9307F0FF2322F404032481003E
:100930008320C10083244100130101016F30502D39
:1009400063000508130101FF232481002322910085
:10095000130405002326110093840500EF301028AE
:10096000832604048327C40303270400232C0402E2
:10097000B387F6021306F0FF2322C4042324E40005
:100980002324C404B386D740B307F7003307D70046
:100990002322F4002326E400639804028327040141
:1009A000639E0702EF30D0268320C100032481001C
:1009B000832441001305100013010101678000002A
:1009C000737004306F00000013050401EFF01FD6B0
:1009D00013054402EFF09FD56FF0DFFC130504010F
:1009E000EF30C04E93071000E31EF5FAEFF05FBA48
:1009F0006FF05FFB63160500737004306F0000003A
:100A0000130101FE232A910023282101232631010D
:100A1000232E1100232C8100930906001389050061
:100A200093040500638E05083305B50213055505CB
:100A3000EF50C00213040500630C05089307450539
:100A40002320F500232E940223202405EF301019D3
:100A5000832604048327C403032704001306F0FF3E
:100A6000B387F602232C04022322C4042324E400C7
:100A70002324C40413050401B386D740B307F70049
:100A80003307D7002322F4002326E400EFF01FCA27
:100A900013054402EFF09FC9EF3090172308340587
:100AA000130504008320C101032481018324410133
:100AB000032901018329C10013010102678000009D
:100AC00013054005EF4090791304050063160500F7
:100AD000737004306F000000232084006FF09FF6D5
:100AE00063160500737004306F0000006376B50074
:100AF000737004306F000000130101FF2324810094
:100B0000130620001384050093050000232611001E
:100B1000EFF05FEE630C0500232C85028320C100FB
:100B20000324810013010101678000007370043009
:100B30006F000000130101FB23261104232481040C
:100B40002322910423202105232E3103232C41034A
:100B5000232A510323286103232671032326C1007E
:100B600063060528638C052693072000639CF60026
:100B70000327C503930710006306F7007370043062
:100B80006F0000001389060093840500130405001C
:100B9000EF300065631A05008327C10063860700F4
:100BA000737004306F000000EF305003032784039C
:100BB0008327C403130B0000930B20009309F0FF5D
:100BC000130A0401930A44026364F710630479234F
:100BD0008327C1006382073663160B00130581016A
:100BE000EF308049EF30D002EF10D074EF30007F4B
:100BF0008327440463943701232204048327840455
:100C00006394370123240404EF3090009305C1005E
:100C100013058101EF30404963160530EF30007C49
:100C2000032784038327C4036304F710EF30407E57
:100C3000EF30C07A832784046346F0026F0000031C
:100C400013850A00EF30802863040500EF3040551B
:100C5000832784049387F7FF2324F40483278404E1
:100C60006356F00083274402E39C07FC23243405E9
:100C7000EF30007AEF308076832744046346F00239
:100C80006F00000313050A00EF30402463040500E1
:100C9000EF300051832744049387F7FF2322F404A5
:100CA000832744046356F00083270401E39C07FC78
:100CB00023223405EF30C075EF20401B130B1000CA
:100CC000EF30C071032784038327C403E370F7F078
:100CD0000326040463040612631A091E0325840014
:100CE00093850400EF401078832784008326040452
:100CF00003274400B387D7002324F40063E4E710FC
:100D00008327840383260400032744029387170064
:100D10002324D400232CF40263000710130544029B
:100D2000EF30C01A930710006318F50E6F004014DF
:100D3000EF30006E8325C10013050A00EF20106C10
:100D4000EF30C069832784046346F0026F0000031C
:100D500013850A00EF30801763040500EF3040442C
:100D6000832784049387F7FF2324F40483278404D0
:100D70006356F00083274402E39C07FC23243405D8
:100D8000EF300069EF308065832744046346F0024A
:100D90006F00000313050A00EF30401363040500E1
:100DA000EF300040832744049387F7FF2322F404A5
:100DB000832744046356F00083270401E39C07FC67
:100DC00023223405EF30C064EF20400AE31805EE1B
:100DD000EFF00FFC130B10006FF09FEE832705045C
:100DE000E38407D8737004306F0000007370043020
:100DF0006F00000003260404631006088327040024
:100E0000638607048327840303274402938717001C
:100E1000232CF402E31407F0EF30805F1305100079
:100E20008320C10403248104832441040329010491
:100E30008329C103032A8103832A4103032B01036E
:100E4000832BC102130101056780000003254400C4
:100E5000EF30C04B8327840303274402232204007E
:100E600093871700232CF402E31A07EAE30605FA36
:100E7000EFF00FF26FF05FFA0325C40093850400D2
:100E8000EF40505E832704040327C4008326040038
:100E9000B307F0403307F7002326E400637ED7044E
:100EA00003274400B307F7002326F40013072000AC
:100EB000832744026304E90403278403130717000C
:100EC000232CE402E38A07F46FF05FE50325C400F6
:100ED00093850400EF401059832704040327C400BE
:100EE00083260400B307F0403307F7002326E4000D
:100EF000E37ED7FA6FF0DFFA8327440203278403E7
:100F0000E30C07FA032784031307F7FF232CE402FB
:100F10000327840313071700232CE402E38E07EE54
:100F20006FF0DFDF13050400EFF05F92EF10107435
:100F3000130500006FF0DFEEEF30804D1305000069
:100F40006FF01FEE130101FF2322910093040500AF
:100F5000130540052324810023261100EF401030A3
:100F600013040500630C0504232C05029307F0FF0E
:100F70002322F5041307100013050501232EE402B4
:100F80002324F40423220400232004002324040047
:100F9000232604002320040423089404EFF00FF90F
:100FA00013054402EFF08FF89306000013060000CB
:100FB0009305000013050400EFF0DFB713050400EC
:100FC0008320C10003248100832441001301010117
:100FD0006780000063040504130101FF23248100DE
:100FE00023229100232611002320210103294500FB
:100FF00013040500EF30C01D930400006304A90230
:101000008320C1000324810013850400032901000B
:1010100083244100130101016780000073700430D4
:101020006F0000008327C400930410009387F7FF2C
:101030002326F400E39607FC930600001306000045
:101040009305000013050400EFF0DFAE6FF05FFBC7
:101050006302050A63880508130101FE232C810041
:10106000232A91002328210123244101232E11004A
:1010700023263101930720009384060013090600FC
:10108000138A050013040500639CF6000327C503BB
:10109000930710006302F70A737004306F000000BA
:1010A000EFF04FE3032784038327C403930905006C
:1010B0006366F7049304000013850900EFF00FE165
:1010C0008320C10103248101138504000329010148
:1010D000832441018329C100032A810013010102F5
:1010E0006780000083270504E38807F673700430E7
:1010F0006F000000737004306F00000003260404CA
:10110000631E060C8327040063860712832784036B
:101110001307F0FF93871700232CF402832784041E
:101120006388E70E832784049304100093871700D5
:101130002324F4046FF05FF8EFF0CFD90327840382
:101140008327C403930905006360F706032604049C
:10115000E30A06FA0325C40093050A00EF40903025
:10116000832704040327C40083260400B307F04048
:101170003307F7002326E4006378D70003274400F1
:10118000B307F7002326F40093072000E390F4F858
:1011900083278403E38C07F6832784039387F7FF71
:1011A000232CF4026FF09FF603260404E30C06F4EC
:1011B0000325C40093050A00EF40D02A83270404C6
:1011C0000327C40083260400B307F0403307F70069
:1011D0002326E400E364D7FA6FF09FFBE39C04F658
:1011E0000325840093050A00EF40D027832784005D
:1011F0008326040403274400B387D7002324F40084
:10120000E3E6E7F0832704002324F4006FF01FF0E7
:101210008327440293041000E38007EA1305440285
:10122000EF20D04AE30A05E8E30809E82320990003
:101230006FF09FE803254400EF30400D23220400A7
:101240006FF0DFEC6302050A83270504638607005D
:10125000737004306F00000083270500638A07085D
:10126000130101FE232C8100232A910013040500A1
:101270002328210123263101232E11001389050083
:10128000EFF04FC5032784038327C40393090500A8
:10129000930400006376F702832784031307F0FFAB
:1012A00093871700232CF40283278404638AE704BE
:1012B0008327840493041000938717002324F404E5
:1012C00013850900EFF08FC08320C1010324810141
:1012D0001385040003290101832441018329C100EE
:1012E0001301010267800000737004306F0000007A
:1012F00083274500E38607F6737004306F00000013
:101300008327440263960700930410006FF05FFB8D
:1013100013054402EF20903BE30805FEE30609FEB7
:10132000930710002320F9006FF01FFE130101FC4A
:10133000232E1102232C8102232A91022328210328
:101340002326310323244103232251032326C100F2
:1013500063060528638C0526938A06009389050099
:1013600013040500EF20D067631A05008327C1002E
:1013700063860700737004306F000000EF300006D2
:10138000832784036394071C8327C10063800710AD
:1013900013058101EF20504E9304F0FF130944021E
:1013A000130A0401EF30C006EF10C078EF300003DD
:1013B000832744046394970023220404832784042E
:1013C0006394970023240404EF3080049305C10044
:1013D00013058101EF20504D63100524EF3000000C
:1013E00083278403638A070AEF308002EF20107F8F
:1013F000832784046346F0026F000003130509008D
:10140000EF20D02C63040500EF209059832784043B
:101410009387F7FF2324F404832784046356F000A2
:1014200083274402E39C07FC23249404EF20507E8E
:10143000EF20D07A832744046346F0026F00000354
:1014400013050A00EF20902863040500EF20505593
:10145000832744049387F7FF2322F404832744045B
:101460006356F00083270401E39C07FC23229404C5
:10147000EF20107AEF10901FEF205076832784031F
:101480006396070C8327C100E39E07F0EF20507896
:10149000130500006F00800FEF2090778327040072
:1014A000638807108325C10013050900EF2000752C
:1014B000EF20D072832784046346F0026F0000039C
:1014C00013050900EF20902063040500EF20504D24
:1014D000832784049387F7FF2324F4048327840459
:1014E0006356F00083274402E39C07FC2324940402
:1014F000EF201072EF20906E832744046346F002C1
:101500006F00000313050A00EF20501C6304050060
:10151000EF201049832744049387F7FF2322F40424
:10152000832744046356F00083270401E39C07FCEF
:1015300023229404EF20D06DEF10501363040508AC
:10154000EF20D06983278403E38E07F29385090097
:10155000130504008324C400EFF00FAC63940A0861
:1015600083278403032704009387F7FF232CF402C7
:1015700063160700EF2010712322A40083270401C3
:1015800063920708EF20D068130510008320C10381
:101590000324810383244103032901038329C10216
:1015A000032A8102832A410213010104678000009B
:1015B000EF20D06203254400EF205045EF20506516
:1015C0006FF05FEEEFE0DFFC6FF09FF7832705041D
:1015D000E38407D8737004306F0000007370043028
:1015E0006F0000008327440223269400E38C07F851
:1015F00013054402EF20900DE30605F8EFE05FF9D4
:101600006FF05FF813050401EF20500C93071000F2
:10161000E31AF5F66FF09FFE13050400EFF00FA339
:10162000EF10D004130500006FF05FF663000506AD
:10163000130101FF2324810023202101232611000F
:10164000232291008324450013890500130405001B
:10165000EF2010386380A4049306000013060900ED
:101660009305000013050400EFF05FCC9307100012
:10167000630CF5028320C100032481008324410010
:101680000329010013010101678000007370043019
:101690006F0000008327C400130510009387170014
:1016A0002326F4006FF01FFD8327C40093871700E3
:1016B0002326F4006FF01FFC630805066386050C03
:1016C000130101FE232C8100232A910023282101EC
:1016D000232631012324410113040500232E110088
:1016E0001309060093890500EFE0DFFE83278403DA
:1016F000130A050093040000639C070213050A0007
:10170000EFE0DFFC8320C101032481011385040085
:1017100003290101832441018329C100032A810097
:101720001301010267800000737004306F00000035
:1017300003260404630406028325C40083274400AF
:10174000B385C5002326B40063E6F50083250400B5
:101750002326B40013850900EF40C050832784037B
:101760001307F0FF9387F7FF232CF4028327440429
:101770006384E702832744049304100093871700CF
:101780002322F4046FF09FF783270504E38A07F20E
:10179000737004306F000000832704016396070014
:1017A000930410006FF09FF513050401EF20007201
:1017B000E30805FEE30609FE930710002320F90065
:1017C0006FF01FFE6306050883270504638A05087A
:1017D00063840708130101FE232C8100232A910052
:1017E000232821012324410113040500232E110085
:1017F00023263101138A0500EFE0DFED8327840300
:101800001309050093040000638E07008329C400B8
:1018100093050A0013050400EFF00F8093041000F5
:101820002326340113050900EFE05FEA8320C1019C
:10183000032481011385040003290101832441014C
:101840008329C100032A810013010102678000007F
:10185000737004306F000000737004306F0000007C
:10186000E38C07FE737004306F0000006316050000
:10187000737004306F000000130101FF2324810006
:101880001304050023261100EF20503503248403A0
:10189000EF2010388320C1001305040003248100C9
:1018A00013010101678000006316050073700430A6
:1018B0006F000000130101FF232611002324810083
:1018C00013040500EF209031832784030324C4030D
:1018D0003304F440EF20D033130504008320C1000B
:1018E00003248100130101016780000063060500E5
:1018F0000325850367800000737004306F000000CB
:1019000063080504978703009387C7E303A747008D
:101910006304E50403A7C7006302E50803A74701C2
:10192000630AE50603A7C7016302E50603A74702AA
:10193000630AE50403A7C7026302E50403A747039C
:10194000630AE50203A7C7036302E5026F400029AB
:10195000737004306F000000130700001317370086
:10196000B387E70023A007006F40402713077000EC
:101970006FF0DFFE130760006FF05FFE130750008B
:101980006FF0DFFD130740006FF05FFD13073000BD
:101990006FF0DFFC130720006FF05FFC13071000EF
:1019A0006FF0DFFB0325C504678000002326B50424
:1019B0006780000003450505678000006308050097
:1019C000032585031335150067800000737004300C
:1019D0006F000000630C0500832785030325C50302
:1019E0003305F5401335150067800000737004302F
:1019F0006F000000978703009387C7D403A70700F1
:101A00006300070403A787006308070403A707010F
:101A10006308070403A787016308070403A70702F5
:101A20006308070403A787026308070403A70703E3
:101A3000630C070403A7870363040704678000009F
:101A40001307000013173700B387E70023A0B70080
:101A500023A2A70067800000130710006FF09FFE0D
:101A6000130720006FF01FFE130730006FF09FFD7B
:101A7000130740006FF01FFD130750006FF09FFC2D
:101A8000130770006FF01FFC130760006FF09FFBDF
:101A900097870300938707CB03A747006300E504FC
:101AA00003A7C7006306E50403A747016306E5042F
:101AB00003A7C7016306E50403A747026306E5041D
:101AC00003A7C7026306E50403A74703630AE50407
:101AD00003A7C7036302A704678000001307000081
:101AE00013173700B387E70023A0070067800000C3
:101AF000130710006FF0DFFE130720006FF05FFE8A
:101B0000130730006FF0DFFD130740006FF05FFD3B
:101B1000130750006FF0DFFC130770006FF05FFCDD
:101B2000130760006FF0DFFB130101FF2324810026
:101B300023229100232021011304050023261100F4
:101B40009384050013090600EF205009032744047D
:101B50009307F0FF6314F70023220404032784048F
:101B60009307F0FF6314F70023240404EF20500AC6
:101B700083278403639A07001306090093850400F2
:101B800013054402EF20C023EF205005832784046F
:101B9000635AF004832744026386070493044402D3
:101BA0006F000002832784049387F7FF2324F40443
:101BB000832784046358F002832744026384070266
:101BC00013850400EF208030E30E05FCEF20405D1C
:101BD000832784049387F7FF2324F4048327840452
:101BE000E34CF0FC9307F0FF2324F404EF205002B1
:101BF000EF20C07E83274404635AF0048327040146
:101C000063860704930404016F00000283274404E1
:101C10009387F7FF2322F404832744046358F002D8
:101C2000832704016384070213850400EF20002A40
:101C3000E30E05FCEF20C056832744049387F7FF8B
:101C40002322F40483274404E34CF0FC9307F0FFC1
:101C50002322F404032481008320C1008324410053
:101C600003290100130101016F20807A6304050438
:101C7000130101FD232E3101232C410123261102E2
:101C8000138A0700232481022322910223202103A7
:101C9000232A510123286101232671012324810174
:101CA000930790009309070063FAE700737004300C
:101CB0006F000000737004306F000000930A05008D
:101CC0009384050013090600938B0600130B08008C
:101CD0006304082C13050006EF3050581304050068
:101CE0006304052A13192900232865031306090034
:101CF0009305500A13050B00EF40C00803C704000A
:101D0000832704031309C9FF230AE40203C704005D
:101D1000338927011379C9FF6306070E83C71400AF
:101D2000A30AF40283C71400638E070C83C7240040
:101D3000230BF40283C724006386070C83C7340097
:101D4000A30BF40283C73400638E070A83C74400E1
:101D5000230CF40283C744006386070A83C7540038
:101D6000A30CF40283C75400638E070883C7640082
:101D7000230DF40283C764006386070883C77400D9
:101D8000A30DF40283C77400638E070683C7840023
:101D9000230EF40283C784006386070683C794007A
:101DA000A30EF40283C79400638E070483C7A400C4
:101DB000230FF40283C7A4006386070483C7B4001B
:101DC000A30FF40283C7B400638E070283C7C40065
:101DD0002300F40483C7C4006386070283C7D400CA
:101DE000A300F40483C7D400638E070083C7E40014
:101DF0002301F40483C7E4006386070083C7F4006B
:101E0000A301F404130B440013050B00A301040405
:101E10002326340323283405232A0404EFE01F93E8
:101E200013058401EFE09F929307A000B387374129
:101E3000232C040423288400232CF400232284026E
:101E400023220404232E040413860B0093850A0026
:101E500013050900EFE0DF882320A40063040A00D3
:101E600023208A007370043017E901001309C96147
:101E70008327090097E401009384C462638C070000
:101E800003A7040083A70400832747049387170050
:101E90002322F70417E701001307C75F8327070012
:101EA0009387170097E6010023A6F65E83A7040038
:101EB000638007108327090017EA0100130A4A6CA0
:101EC000639C070083A7040083A7C70263E6F900A9
:101ED00097E7010023A8875C97E701009387C7591C
:101EE00003A7070097E601009386465A8327C4029A
:101EF00083A606001307170017E60100232EE656F7
:101F00002324E40463F6F60017E701002320F758C2
:101F100013074001B387E70293050B003305FA006E
:101F2000EFE05F83832709006388070083A704002D
:101F300083A74704639E0708832709001304100042
:101F4000638A070083A7040083A7C70263F43701ED
:101F5000EFE00FE4130504008320C1020324810293
:101F600083244102032901028329C101032A81013B
:101F7000832A4101032B0101832BC100032C810023
:101F8000130101036780000013050B00EF301045BB
:101F90001304F0FF6FF01FFC13152600EF30102C18
:101FA000130B0500E31805D21304F0FF6FF09FFA3E
:101FB00097E7010023A8874E032707009307100027
:101FC000630AF70217EA0100130A8A5B6FF0DFF079
:101FD00003A7040083A60400832747049387F7FF21
:101FE0002322F70483A74604E39807F473600430C0
:101FF0006FF09FF4930A000017EA0100130A4A5891
:10200000130C4001930BA00033858A03938A1A00B6
:102010003305AA00EFE08FF1E3987AFF97EB010018
:10202000938B8B6213850B00EFE04FF097EA010072
:10203000938ACA6213850A00EFE04FEF17E50100AB
:1020400013050563EFE08FEE17E5010013058563C7
:10205000EFE0CFED17E5010013050564EFE00FEDAC
:1020600097E7010023AE774397E7010023A8574382
:102070006FF09FE6130101FF232481002326110046
:1020800023229100232021011304050073700430E2
:1020900097E401009384443F83A70400639E0710E4
:1020A0006318040097E701009387C73F03A4070064
:1020B0001309440013050900EFE00FF2832784029F
:1020C0006386070013058401EFE00FF19305090013
:1020D00017E501001305055BEFE0CFE797E7010087
:1020E0009387873B03A7070097E701009387C738CB
:1020F00083A707001307170097E6010023AEE63811
:1021000003A704009387170097E6010023A6F6367D
:10211000630C070097E701009387C73803A7070000
:1021200003274704631C070E83A70400638A07067E
:1021300097E701009387073703A70700630287101B
:102140007370043003A704006318070817E7010041
:10215000130707358326070083A606006392060A45
:102160001307F0FF97E6010023A6E63003A704005B
:102170006308070203A70700032747046302070257
:1021800003A7070083A60700832747049387F7FF69
:102190002322F70483A74604639407007360043086
:1021A0008320C1000324810083244100032901000E
:1021B000130101016780000097E701009387872ED4
:1021C00003A7070083A70700832747049387170007
:1021D0002322F7046FF0DFEC83A6070003A70700B4
:1021E00003A746041307170023A2E60417E701001C
:1021F0001307072B8326070083A60600E38206F653
:10220000032707000327C7000327C700032747004A
:1022100097E6010023A0E6266FF05FF503A707000D
:1022200083A60700832747049387F7FF2322F70439
:1022300083A74604E39A07EE736004306FF0DFEE85
:1022400097E701009387C72283A7070063860700EB
:10225000737004306F000000032481008320C100EC
:102260008324410003290100130101016FE04FB2F3
:102270006304050C17E701001307C7228326070034
:10228000930700006386A60A130101FF23261100AD
:1022900023248100232291007370043097E601000B
:1022A0009386861E83A70600638C0700032607001B
:1022B0008327070083274604938717002322F60409
:1022C00083A70600930405000324450163880700E3
:1022D0008327070083A747046394070697E7010055
:1022E0009387071C83A70700638C870697E7010085
:1022F0009387C71A83A707006384870697E70100BF
:10230000938787396306F40497E70100938787373B
:10231000630CF402930710008320C10003248100A2
:102320008324410013850700130101016780000029
:102330001385070067800000737004306F00000091
:10234000EF50504E6FF09FF9930740006FF0DFFCA5
:1023500083A7840293B71700938727006FF0DFFBF2
:10236000930720006FF05FFB7370043097E7010064
:102370009387871103A70700631607026304050408
:1023800083A707000325C502638C070097E70100B8
:102390009387471103A7070003274704631C07021D
:1023A0006780000017E701001307C70F83260700A7
:1023B0000327070003A746041307170023A2E60418
:1023C000E31005FC17E701001307C70D03250700FD
:1023D0006FF01FFB03A7070083A6070083274704AE
:1023E0009387F7FF2322F70483A74604E39A07FAAB
:1023F0007360043067800000130101FF2324810013
:102400001304050023261100EFE0CFAC631804008D
:1024100097E701009387070903A407000324C40278
:10242000EFE0CFAA8320C10013050400032481003C
:1024300013010101678000009307900063F6B70065
:10244000737004306F000000130101FE232C810023
:10245000232E1100232A9100232821012326310154
:1024600023244101130405007370043017E90100AF
:10247000130989018327090063920710630004127E
:1024800083270405638EF50A17E701001307870108
:1024900063F0B70283260700638E861203270700C6
:1024A0008324C702B3B4950093C414006F000001E5
:1024B00083240700B384844093B414000327C40228
:1024C0006386E70E832784012328B40463C80700CA
:1024D0009307A000B385B740232CB40093172700BF
:1024E000B387E7000327440197E90100938949096D
:1024F00093972700B387F9006310F704130A440089
:1025000013050A00EFE04FAD17E70100130707F8C6
:102510008327C402032707006376F70017E701004B
:102520002326F7F613074001B387E70293050A0055
:102530003385F900EFE00FA263840400EFE04F85DC
:1025400083270900638C070097E70100938787F5CD
:1025500083A7070083A74704639E07048320C10164
:102560000324810183244101032901018329C1003E
:10257000032A8100130101026780000097E7010030
:10258000938747F203A7070083A707008327470421
:10259000938717002322F704E31404EE97E7010062
:1025A000938747F003A407006FF09FED2326B40242
:1025B0006FF05FF1032481018320C1018324410175
:1025C000032901018329C100032A810013010102AB
:1025D0006F505025930400006FF05FEE630A05080A
:1025E000130101FE232A910097E40100938484EBF8
:1025F00083A70400232E1100232C8100232821010E
:10260000232631016388A7047370043017E90100A1
:10261000130989E783270900638C070003A70400D7
:1026200083A7040083274704938717002322F70416
:102630000327450197E7010093870706630EF7021A
:10264000832709006388070083A7040083A7470442
:10265000639E07088320C101032481018324410173
:10266000032901018329C1001301010267800000D1
:10267000737004306F0000008327850217E70100A4
:10268000130707FFE38EE7FAE39C07FA9309450077
:102690001304050013850900EFE00F9417E701000C
:1026A0001307C7DE8327C402032707006376F700FA
:1026B00017E70100232CF7DC13074001B387E7027B
:1026C00017E501001305C5EB938509003305F500F7
:1026D000EFE04F8883A704000327C40283A7C70243
:1026E000E360F7F6EFD0DFEA6FF09FF50324810196
:1026F0008320C10183244101032901018329C100F1
:10270000130101026F50101263020506130101FE4E
:10271000232C8100232A9100232821011304050082
:10272000232E110023263101EFD0DFFA03274401C5
:1027300097E70100938747F613090500930400000B
:10274000630AF70213050900EFD05FF88320C10187
:10275000032481011385040003290101832441011D
:102760008329C100130101026780000073700430E7
:102770006F0000008327840217E50100130545EF71
:10278000E382A7FCE39007FC97E70100938747CE1D
:1027900083A707006394070697E70100938787D014
:1027A00083A707008324C4029309440083A7C702B8
:1027B00013850900B3B4F400EFE00F8217E70100BE
:1027C0001307C7CC8327C4020327070093C4140050
:1027D0006376F70017E70100232AF7CA13074001C1
:1027E000B387E70217E50100130585D99385090032
:1027F0003305F500EFD01FF66FF0DFF49305840189
:10280000EFD05FF56FF01FF4130101FE37150000E4
:10281000232E1100232C8100232A9100232821013B
:102820002326310123244101232251012320610168
:10283000EF30C0226308052293040500130500064B
:10284000EF30C0211304050063040526371600008D
:102850009305500A2328950213850400EF30805217
:1028600083240403B71700009387C7FFB384F400E1
:10287000B7474C4593879744130A4400232AF40230
:1028800013050A00230C0402A301040423260402F6
:1028900023280404232A0404EFD05FEB13058401EA
:1028A000EFD0DFEA9307A000232C040493F4C4FFC5
:1028B00023288400232CF4002322840223220404EE
:1028C000232E040413060000971500009385C5EA23
:1028D00013850400EFD0DFE02320A40073700430E0
:1028E00017E90100130949BA8327090097E4010099
:1028F000938444BB638C070003A7040083A70400F0
:1029000083274704938717002322F70417E7010062
:10291000130747B8832707009387170097E601003E
:1029200023AAF6B683A704006388070A8327090051
:1029300097E901009389C9C4639C070083A7040039
:1029400083A7C7026396070097E7010023AC87B40B
:1029500097E70100938747B203A7070097E60100B6
:102960009386C6B28327C40283A606001307170006
:1029700017E601002322E6B02324E40463F6F60000
:1029800017E701002324F7B0139527003305F5005E
:102990001315250093050A003385A900EFD09FDBAE
:1029A000832709006388070083A7040083A74704DF
:1029B000639E070C832709006384070083A7040034
:1029C000EF20500693071000630AF510631C0508FA
:1029D000737004306F00000097E7010023A487ACF8
:1029E000032707009307100097E90100938949B96D
:1029F000E310F7F6938A090017EB0100130BCBC421
:102A000013850A00938A4A01EFD05FD2E31A5BFF75
:102A100017E50100130545C3EFD05FD197EA010028
:102A2000938ACAC313850A00EFD05FD017E501006F
:102A3000130505C4EFD09FCF17E50100130585C42A
:102A4000EFD0DFCE17E50100130505C5EFD01FCE8F
:102A500097E7010023A667A597E7010023A057A5E4
:102A60006FF01FEF8320C101032481018324410102
:102A7000032901018329C100032A8100832A41001F
:102A8000032B0100130101026780000003A704006B
:102A900083A60400832747049387F7FF2322F704C4
:102AA00083A74604E39807F0736004306FF09FF04B
:102AB000032481018320C101032901018329C1006D
:102AC000032A8100832A4100032B0100138504009F
:102AD00083244101130101026F30401073700430F0
:102AE0009307F0FF17E701002326F79803248101DD
:102AF00097E7010023AAA7988320C10183244101FD
:102B0000032901018329C100032A8100832A41008E
:102B1000032B010097E7010023AC07961301010284
:102B20006FD05F8C7370043097E7010023AE079479
:102B30006FD09F9D17E70100130787938327070036
:102B4000938717002320F70067800000737004301C
:102B500097E701009387479303A7070063180702CD
:102B600017E701001307C7920325070083A7070093
:102B7000638C070097E701009387C79203A70700BC
:102B800003274704631407026780000017E701006A
:102B900013074791832607000327070003A746046E
:102BA0001307170023A2E6046FF09FFB03A707009B
:102BB00083A60700832747049387F7FF2322F704A0
:102BC00083A74604E39207FC73600430678000002B
:102BD000130101FF2326110023248100EFD09FAFB2
:102BE00097E701009387C78A03A40700EFD01FAEC1
:102BF0008320C10013050400032481001301010197
:102C00006780000097E701009387C78803A5070046
:102C100067800000130101FD232611022324810295
:102C20002322910223202103232E3101232C410151
:102C3000232A5101232861012326710197E701000E
:102C40009387078383A70700639A070617E70100A6
:102C500013070784832707009387170097E601006F
:102C600023A8F682832A0700638A0A0A97E70100ED
:102C70009387478083A707009304000063FEFA0A46
:102C800097E901009389C98F17EA0100130A8A8125
:102C900083270A009306100003A7C7029317270093
:102CA000B387E70093972700B389F90083A709004A
:102CB00063F4F602930410006F00000297D701003E
:102CC0009387477C83A7070093040000938717002E
:102CD00017D701002328F77A97D701009387477AFF
:102CE00083A7070063840700930410008320C102B8
:102CF0000324810213850400032901028324410275
:102D00008329C101032A8101832A4101032B010187
:102D1000832BC100130101036780000017D4010059
:102D2000130404788327040083A707006388070C33
:102D3000737004306F00000017D401001304447650
:102D400097E901009389C98317DA0100130A8A758C
:102D500017DB0100130B8B738327040083A7070085
:102D6000638007088327040083A7C70003A9C7005F
:102D700083274900930B490013850B0063EAFA0689
:102D8000EFD09FA58327890213058901638407007B
:102D9000EFD09FA48327C90203270B0093850B0064
:102DA000139527003305F500131525003385A90079
:102DB0006376F70017D70100232AF76CEFD09F99AD
:102DC00083270A000327C90283A7C702E366F7F82F
:102DD000832704009304100083A70700E39407F8F7
:102DE0009307F0FF17D701002326F7686FF05FEA1B
:102DF00017D701002320F7686FF09FE917D701006C
:102E00001307C769832704000327070097D601002B
:102E100023A8E66817D701002322F76897D7010097
:102E20009387C76583A707009387170017D701000B
:102E30002326F7648327040083A70700639A07000B
:102E40009307F0FF17D701002326F7626FF01FE208
:102E50008327040083A7C70083A7C70083A7470071
:102E600017D701002328F7606FF05FE097D70100C4
:102E70009387076003A70700631607007370043089
:102E80006F000000130101FE232E1100232C81008E
:102E9000232A9100232821012326310123244101E3
:102EA00023225101232061017370043097D4010063
:102EB0009384845D03A704006310071203A707002F
:102EC0001307F7FF97D6010023A4E65A83A707004C
:102ED000639E070A97D701009387C75B83A7070004
:102EE0006386070A97DA0100938A8A6917DA010074
:102EF000130ACA5917D901001309C95A93091000B6
:102F00006F00C0013385EA00EFD0DF84832709001A
:102F10000327C40283A7C7026374F70683A70A0FB7
:102F20006380070E83A7CA0F03A4C700130584019B
:102F3000EFD09F8A130B440013050B00EFD0DF89FD
:102F40008327C40283260A0093050B0013952700EC
:102F50003305F50013152500130705003385AA0076
:102F6000E3F2F6FA17D701002322F752EFD08FFED3
:102F7000832709000327C40283A7C702E360F7FA87
:102F800097D7010023AE374F6FF05FF913040000AD
:102F900083A70400638C070097D7010093878750AD
:102FA00083A7070083A74704639807041305040059
:102FB0008320C101032481018324410103290101EC
:102FC0008329C100032A8100832A4100032B0100C9
:102FD000130101026780000017D701001307874C17
:102FE000832607000327070003A7460413071700DB
:102FF00023A2E6046FF09FECEF50C0026FF01FFBBE
:1030000017D401001304044883270400638C0702CB
:10301000832704001309100063860702EFF09FBFA7
:103020006306050097D7010023AC274583270400DA
:103030009387F7FF17D701002326F744832704005F
:10304000E39E07FC97D701009387874303A70700F8
:1030500093071000E31CF7F2EFD08FD31304100096
:103060006FF01FF36304050263960500737004306C
:103070006F00000017D701001307873F8327070061
:10308000638A0700737004306F00000073700430AF
:103090006F000000130101FF23248100232611008B
:1030A00083260700032705009386160017D6010024
:1030B0002320D63C97D601009386863D83A6060042
:1030C0003304B7002320850063F0E6046372E40252
:1030D00063F0860297D701009387C73C03A50700DA
:1030E00013054500EFD04FEF13050400EF40106BC0
:1030F000EFF0DFD7630E05008320C10003248100B9
:103100001301010167800000E366E4FC6FF05FFCDF
:10311000032481008320C100130101016FD04FC738
:10312000630E050017D701001307873483270700B4
:1031300063880700737004306F0000006FD04FC5C4
:10314000130101FF23261100232481000327070018
:10315000930705001307170097D6010023AAE6304E
:1031600097D601009386063417D70100130747321C
:103170000327070003A506003304F70013054500E5
:10318000EFD08FE513050400EF405061EFF01FCE44
:10319000631A0500032481008320C100130101018B
:1031A0006FD00FBF8320C1000324810013010101F0
:1031B00067800000130101FF2324810023261100F2
:1031C00097D701009387C72A83A70700130400003D
:1031D0009387170017D70100232CF72897D70100F2
:1031E0009387472B83A7070063EEF51417DE0100D2
:1031F000130ECE4497D201009382C237130400000D
:1032000013070000930F10001303500A6F00C00053
:10321000130ECEFE6384C20F83278EFF9306070032
:10322000E38807FE8327CEFF83A74700232EFEFEF9
:103230006386C71303AFC70083A747003307E500C2
:10324000930E0000232EFEFE6380C70983A8C700EB
:1032500093874803232017012322F70083A78804BC
:103260002326F7012324F70083A7C8022328F700A9
:1032700083A70805232C0700232AF70003A80803C7
:103280008347080063986704930708009387170033
:1032900083C60700B3850741E38A66FE93D5250000
:1032A0009395050193D50501231EB700938E1E004B
:1032B00013070702630A1F038327CEFF83A7470074
:1032C000232EFEFEE394C7F983274E00232EFEFE35
:1032D0006FF0DFF793050000231EB700938E1E00EA
:1032E00013070702E31A1FFD3304D4011317540018
:1032F000130ECEFE93060700E390C2F397D70100AA
:103300009387071A03AE070083270E006396071200
:1033100097D701009387871803AE070083270E0015
:10332000639A071C17DE0100130E8E2583274E10AB
:10333000639C070283278E11639C072663040600A3
:1033400023200600EFF09FB2130504008320C10084
:1033500003248100130101016780000083274E00D0
:10336000232EFEFE6FF01FED83278E1017DF010066
:10337000130FCF3183A7470017D701002326F7305B
:103380006386E73D83A2C70083A74700B306D50045
:10339000930E000017D701002328F72E930F40004B
:1033A0001303500A6382E70983A8C7009387480381
:1033B00023A0160123A2F60083A7880423A6F60102
:1033C00023A4F60083A7C80223A8F60083A7080554
:1033D00023AC060023AAF60003A8080383470800CD
:1033E000639A6732930708009387170003C70700A3
:1033F000B3850741E30A67FE93D72500939707013A
:1034000093D70701239EF600938E1E009386060233
:10341000638C123183278E1083A7470017D70100D2
:103420002324F726E392E7F983270E1117D701002B
:10343000232CF7246FF05FF783274E00130F8E00C5
:1034400083A647002322DE006380E633B307E5004E
:1034500003A7460083A2C600930E00002322EE00BD
:10346000930F20001303500A6300EF088328C7005E
:103470001387480323A0170123A2E70003A78804AA
:1034800023A6F70123A4E70003A7C80223A8E700A7
:1034900003A7080523AC070023AAE70003A8080335
:1034A00003470800631E672213070800130717006D
:1034B00083460700B3050741E38A66FE13D725005C
:1034C0001317070113570701239EE700938E1E0071
:1034D000938707026380122383264E0003A74600CA
:1034E0002322EE00E314EFF80327CE002322EE00A0
:1034F0006FF0DFF783274E00130F8E0083A747007E
:103500002322FE00638CE72583A2C70083A7470020
:10351000B306D500930E00002322FE00930F200077
:103520001303500A6300FF0883A8C700938748036A
:1035300023A0160123A2F60083A7880423A6F60180
:1035400023A4F60083A7C80223A8F60083A70805D2
:1035500023AC060023AAF60003A80803834708004B
:1035600063986714930708009387170003C7070041
:10357000B3850741E30A67FE93D7250093970701B8
:1035800093D70701239EF600938E1E0093860602B2
:10359000638A121383274E0083A747002322FE006D
:1035A000E314FFF88327CE002322FE006FF0DFF73D
:1035B0008327CE1197DE0100938E8E0E83A74700DE
:1035C00017D70100232CF70C638AD71783AFC700E6
:1035D00083A747003307D5001303000097D60100E7
:1035E00023AEF60A130F3000930220009308500A0E
:1035F0006388D70903A5C700930745032320A700C5
:103600002322F700832785042326E7012324F700DC
:103610008327C5022328F7008327850263840700D8
:103620002326570083270505232C0700232AF700AC
:103630000328050383470800639C170593070800C8
:103640009387170083C60700B3850741E38A16FFF7
:1036500093D725009397070193D70701231EF700FF
:103660001303130013070702638EAF028327CE11E3
:1036700083A7470097D6010023A2F602E39CD7F761
:1036800083274E1297D6010023AAF6006FF09FF60B
:1036900093070000231EF70013031300130707020C
:1036A000E396AFFC33046400E31C06C86FF09FC9C7
:1036B00093070000239EF600938E1E009386060259
:1036C000E39A12ED17DE0100130E8EEB83274E10E6
:1036D0003304D40193165400E38E07C46FF0DFC89F
:1036E00013070000239EE700938E1E0093870702B6
:1036F000E39412DF97D70100938747DA03AE070000
:103700003304D4019316540083270E00E38C07C0C2
:103710006FF05FDE93070000239EF600938E1E007D
:1037200093860602E39812CF83278E113304D401C7
:1037300093165400E38407C06FF09FE783274E126F
:1037400017D70100232CF7F46FF05FE883270E11E1
:1037500017D70100232AF7F26FF0DFC28327CE00CC
:103760002322FE006FF05FDA8326CE002322DE00E4
:103770006FF0DFCD130101FD2322910223202103ED
:10378000232E3101232C4101232A510123286101D9
:1037900023267101232611022324810297D90100D7
:1037A000938909CD17D90100130989DD17DA0100C2
:1037B000130A8ACD97DA0100938ACACE97DB0100FB
:1037C000938B4BCD97D40100938404CD130B100041
:1037D0006F00000283A70900032449109387170094
:1037E00017D701002326F7C8EFF04FE8631E040047
:1037F00083A70400E39007FE83270900E37AFBFE1A
:10380000EFC01FD96FF0DFFE7370043083270A000A
:10381000639E07048327091103A4C700130544000E
:10382000EFC09FFB83A70B009387F7FF17D701001B
:103830002322F7C683A704009387F7FF17D7010059
:10384000232CF7C483270A006388070083A70A0094
:1038500083A747046398070203250403EF20003879
:1038600013050400EF2080376FF09FF803A70A00CC
:1038700083A70A0083274704938717002322F704AE
:103880006FF05FF903A70A0083A60A0083274704A5
:103890009387F7FF2322F70483A74604E39E07FAE2
:1038A000736004306FF05FFB97D70100938747BCCC
:1038B00083A707006396070E130101FF232611005B
:1038C00097D7010023AE07BA17D70100130787BDAA
:1038D00083270700B7A6A5A59386565A83A7070393
:1038E00083A50700639ED50003A64700631AB600B0
:1038F00083A687006396C60083A7C700638AD700A4
:10390000032507008325070093854503EF30807664
:1039100097D60100938686B703A6060017D7010045
:10392000130707C66F00000283A70600638207081B
:1039300083A706009387F7FF17D601002328F6B464
:1039400003A6060093172600B387C70093972700A6
:10395000B307F70083A70700E38807FC03A6060068
:1039600093172600B387C70093972700B305F70086
:1039700083A6450093878700B307F70083A6460018
:1039800023A2D500638AF60283A7C6008320C10064
:1039900017D701002328F7B0130101016780000049
:1039A0009307100017D70100232CF7AC67800000A5
:1039B000737004306F000000930740013306F60275
:1039C00083A646003307C7002322D7006FF0DFFB32
:1039D000130101FE23282101232E1100232C810035
:1039E000232A910023263101130905007370043046
:1039F00097D40100938444A983A7040017D401003D
:103A0000130444AA639C070C6314090003290400EF
:103A10009309490013850900EFC01FDC8327890241
:103A20006386070013058901EFC01FDB938509003A
:103A300017D50100130545C6EFC0DFD183A70400E9
:103A4000638807008327040083A747046394070A59
:103A5000832704006384270D83A70400638207067D
:103A60007370043083A704006398070E97D7010092
:103A7000938707A303A70700032707006310070C1A
:103A80009307F0FF17D701002326F79E83A70400B2
:103A9000638807028327040083A747046382070221
:103AA0000327040083260400832747049387F7FF36
:103AB0002322F70483A7460463940700736004304D
:103AC0008320C101032481018324410103290101D1
:103AD0008329C1001301010267800000032704004D
:103AE0008327040083274704938717002322F704C2
:103AF0006FF09FF103270400832604008327470407
:103B00009387F7FF2322F70483A74604E39207F481
:103B10007360043083270400E39027F583A7040033
:103B20006382070697D701009387879483A70700CE
:103B30006388070A737004306F00000083A70700D2
:103B400083A7C70083A7C70083A7470017D7010033
:103B50002322F7926FF09FF30327040083270400CA
:103B600083274704938717002322F70497D7010080
:103B70009387079303A7070003270700E30207F0D3
:103B80006FF0DFFB97D701009387C79017D701002D
:103B90001307079F83A70700032787116314F70202
:103BA0008320C1010324810197D7010023AC078E34
:103BB00083244101032901018329C100130101026A
:103BC00067800000032481018320C1018324410117
:103BD000032901018329C100130101026FF0DFCC29
:103BE000032481018320C1018324410103290101B0
:103BF0008329C100130101026FC09F996306050A62
:103C0000130101FF2322910097D40100938484893A
:103C1000232021011389050083A504002326110018
:103C20002324810093858501EFC0DFB503A504003F
:103C300013054500EFC05FBA9307F0FF630AF9066A
:103C400097D701009387C78403A4070003A7040044
:103C500083A707003304240123228700636EF40640
:103C600097D701009387C78303A5070083A50400A6
:103C700093854500EFC01FB197C701009387877FE9
:103C800083A707006376F40097C7010023A4877E0B
:103C90008320C10003248100832441000329010003
:103CA0001301010167800000737004306F00000091
:103CB00083A50400032481008320C10083244100E4
:103CC0000329010017D501001305059D93854500C3
:103CD000130101016FC01FA897C701009387077CDC
:103CE00003A507000324810083A504008320C100ED
:103CF000832441000329010093854500130101013C
:103D00006FC05FA8630E050097C7010093874776D1
:103D100083A70700639A0700737004306F000000E8
:103D2000737004306F000000130101FF2322910023
:103D300097C401009384047703A7040093870500C8
:103D400083A50400B7060080B3E7D700232611003F
:103D500023248100232CF70093858501130406009A
:103D6000EFC05F9F03A5040013054500EFC0DFA669
:103D70009307F0FF6304F40297C70100938747712C
:103D800003A507008320C10083244100330585007B
:103D900003248100130101016F40402083A504002A
:103DA000032481008320C1008324410017D5010032
:103DB0001305858E93854500130101016FC09F99FE
:103DC0006308050A130101FF2322910097C4010033
:103DD0009384446D232021011389050083A50400E9
:103DE00023261100232481009385850113040600F6
:103DF000EFC05F9603A5040013054500EFC0DF9DEB
:103E000093071000630AF40697C701009387476879
:103E100003A4070003A7040083A7070033042401B9
:103E200023228700636EF40697C7010093874767D4
:103E300003A5070083A5040093854500EFC09F9468
:103E400097C701009387076383A707006376F40091
:103E500097C7010023A087628320C100032481004B
:103E60008324410003290100130101016780000040
:103E7000737004306F00000083A5040003248100E8
:103E80008320C100832441000329010017D50100CC
:103E90001305858093854500130101016FC09F8B39
:103EA00097C701009387875F03A50700032481005C
:103EB00083A504008320C10083244100032901005D
:103EC00093854500130101016FC0DF8B130101FFD2
:103ED0002326110023248100232291008327C5007B
:103EE00003A4C7006304040A930484011385040037
:103EF000EFC09F8E97C701009387875783A707005E
:103F0000639A07089304440013850400EFC0DF8C14
:103F100097C70100938787570327C40283A7070029
:103F200063F6E70097C7010023A2E756931727001F
:103F3000B387E7009397270017C501001305456471
:103F4000938504003305F500EFC0DF8097C70100BB
:103F50009387475583A707000327C4021305000072
:103F600083A7C70263FAE7009307100017C7010091
:103F70002328F750130510008320C100032481007B
:103F80008324410013010101678000007370043035
:103F90006F0000009385040017C501001305456DEF
:103FA000EFC04FFB6FF09FFA97C701009387474C14
:103FB00083A7070063960700737004306F0000004A
:103FC000130101FF232611002324810023229100E5
:103FD000B70700800324C500B3E7F5002320F500F0
:103FE00063080408EFC04FFF9304440013850400E6
:103FF000EFC08FFE97C70100938747490327C4028C
:1040000083A7070063F6E70097C7010023A0E748EE
:1040100093172700B387E7009397270017C5010080
:10402000130505563305F50093850400EFC08FF2A4
:1040300097C701009387074783A707000327C40298
:104040001305000083A7C70263FAE7009307100077
:1040500017C701002326F742130510008320C10073
:1040600003248100832441001301010167800000C3
:10407000737004306F0000006304050297C70100ED
:104080009387C73F03A7070097C70100938747405F
:1040900083A707002320E5002322F50067800000A6
:1040A000737004306F0000006304050E638E050C0E
:1040B000130101FF232611002324810013070500AB
:1040C0007370043097C801009388083C83A70800E8
:1040D0006380070297C701009387C73C83A6070048
:1040E00083A7070083A746049387170023A2F6043B
:1040F00017C301001303C33983A705000326030078
:104100009306F0FF130400006388D70417CE010064
:10411000130ECE3603250E00032807008326470022
:104120006306A800130410006378D6023308D64053
:10413000130410006372F80203250E00B387C74012
:1041400003260300B387D70023A0F5002320A70090
:104150002322C7001304000083A70800638C070014
:1041600097C701009387073483A7070083A74704F5
:1041700063940702130504008320C1000324810017
:104180001301010167800000737004306F000000AC
:10419000737004306F000000EF30D0686FF09FFD47
:1041A0009307100017C70100232CF72C678000002D
:1041B000630605000325C5046780000013050000A1
:1041C00067800000630405002326B50467800000B3
:1041D00097C701009387072D03A50700678000009C
:1041E00097C701009387472A83A70700130510008C
:1041F000638C070097C701009387872703A50700F3
:10420000133515001315150067800000630C0508B1
:10421000130101FE232A910097C40100938484288E
:1042200083A70400232E1100232C810023282101C1
:10423000232631010327C50283A7C7026376F7044B
:104240008327850163CC070083A7040083A6C702E8
:104250009307A000B387D740232CF50093172700BE
:10426000B387E7000327450117C901001309493146
:1042700093972700B307F9006308F70283A70400A8
:1042800083A7C7022326F5028320C10103248101ED
:1042900083244101032901018329C1001301010283
:1042A0006780000067800000930945001304050043
:1042B00013850900EFC04FD283A7040017C7010080
:1042C0001307C71C0327070083A7C7022326F4028E
:1042D0006376F70017C70100232AF71A1395270002
:1042E0003305F50003248101131525008320C10146
:1042F00083244101938509003305A9008329C10066
:1043000003290101130101026FC0CFC46306050236
:10431000130101FF23261100232481002322910091
:1043200097C701009387071803A40700630AA40036
:10433000737004306F0000001305000067800000F8
:104340008327440563960700737004306F000000F4
:104350008326C402032704059387F7FF232AF40466
:104360006384E600638E0700130500008320C1000C
:1043700003248100832441001301010167800000B0
:104380009304440013850400EFC00FC58327040580
:1043900017C701001307870F832607001307A00024
:1043A0003307F7402326F402232CE40063F6F600DB
:1043B00017C70100232CF70C13074001B387E7024E
:1043C00017C501001305C51B938504003305F500CF
:1043D000EFC04FB8130510006FF05FF97370043031
:1043E00097C701009387470A83A7070063800702E6
:1043F00097C701009387070B03A7070083A7070050
:1044000083274704938717002322F704678000005F
:1044100097C701009387470783A70700638C0702AC
:1044200097C701009387070803A7070003274704DE
:104430006302070203A7070083A607008327470438
:104440009387F7FF2322F70483A7460463940700AA
:10445000736004306780000097C70100938787046A
:1044600003A6070083A6070003A707009307A00081
:1044700083A6C60203258601B387D740232CF70005
:104480006780000097C701009387C70103A7070053
:10449000630A070083A6070003A746051307170052
:1044A00023AAE60403A5070067800000130101FDAD
:1044B0002320210323261102232481022322910297
:1044C000232E3101130905007370043097C40100D5
:1044D000938484FB83A7040017C40100130484FCA5
:1044E000639E070A8327040083A78705639A070052
:1044F000832704001307100023AEE704639A050E18
:1045000083A70400638807008327040083A7470468
:10451000639A07147370043083A70400639407063A
:104520008327040003A587056308050063020904C7
:104530008327040023AC07048327040023AE070469
:1045400083A70400638807008327040083A7470428
:10455000639207068320C10203248102832441025F
:10456000032901028329C1011301010367800000AF
:1045700003270400832787059387F7FF232CF7047D
:104580006FF09FFB03270400832704008327470461
:10459000938717002322F7046FF09FF80327040086
:1045A0008327040083274704938717002322F704F7
:1045B0006FF05FF30327040083260400832747047A
:1045C0009387F7FF2322F70483A74604E39407F8B1
:1045D000736004308320C1020324810283244102DA
:1045E000032901028329C10113010103678000002F
:1045F000032504002326B10013054500EFC0CF9D1D
:104600008325C1009307F0FF6380F50897C7010079
:10461000938707E883A907000327040083A70700FF
:10462000B389B9002322370163ECF90697C701006B
:10463000938707E703A507008325040093854500BA
:10464000EFC04F9497C701009387C7E283A7070085
:1046500063F6F90097C7010023AE37E1EFB05FF3CF
:104660006FF01FEA03270400832604008327470412
:104670009387F7FF2322F70483A74604E39C07E808
:10468000736004306FF01FE98325040017C5010033
:104690001305850093854500EFC0CF8B6FF01FFC9D
:1046A00097C70100938787DF03A5070083250400D0
:1046B00093854500EFC00F8D6FF05FFA130101FD88
:1046C00023202103232E31012326110223248102DA
:1046D00023229102232C410113890500930906002E
:1046E0007370043097C40100938404DA83A7040034
:1046F00017C40100130404DB639C071403270400A0
:10470000930720000327C7056304F70283270400EB
:104710001345F5FF03A787053375E50023ACA70410
:10472000832704001307100023AEE704639A060AE8
:1047300083A70400638807008327040083A7470436
:10474000639407167370043083A70400639E070602
:10475000638809008327040083A7870523A0F90045
:104760000327040093071000130500000327C70563
:10477000630EF700832704001349F9FF13051000A7
:1047800003A787053379E90023AC270583270400B5
:1047900023AE070483A7040063880700832704006F
:1047A00083A747046392070C8320C102032481027C
:1047B00083244102032901028329C101032A8101C3
:1047C000130101036780000003270400832704000E
:1047D00083274704938717002322F7046FF05FF7BE
:1047E000032504002326D10013054500EFB0DFFEAA
:1047F0008326C1009307F0FF638AF60C97C7010078
:10480000938707C903AA07000327040083A70700AB
:10481000330ADA00232247016368FA0C97C70100C4
:10482000938707C803A507008325040093854500E7
:10483000EFB05FF597C701009387C7C383A7070051
:104840006370FA0A97C7010023A647C36F004009A7
:104850000327040083270400832747049387170056
:104860002322F7046FF09FE9032704008326040046
:10487000832747049387F7FF2322F70483A746047F
:10488000E39407F2736004308320C10203248102A1
:1048900083244102032901028329C101032A8101E2
:1048A000130101036780000003270400832604002E
:1048B000832747049387F7FF2322F70483A746043F
:1048C000E39207E8736004306FF0DFE783250400AC
:1048D00017C50100130545DC93854500EFB09FE740
:1048E000EFB01FCB6FF0DFE497C70100938707BBE2
:1048F00003A507008325040093854500EFB09FE8DA
:104900006FF01FFE630A050C130101FF232611003F
:10491000232481002322910023202101737004307D
:1049200097C40100938444B683A7040063960708E4
:10493000638606008327850523A0F60093070600FB
:10494000930620000326C505232ED50413870500F2
:10495000130405006382D70A63F4F6089305300058
:104960006388B700930540006396B700630CD610C8
:10497000232CE40493071000630CF60813041000C2
:1049800083A70400638C070097C70100938787B152
:1049900083A7070083A7470463980706130504004D
:1049A0008320C100032481008324410003290100E6
:1049B000130101016780000097C70100938787AE4C
:1049C00003A7070083A707008327470493871700DF
:1049D0002322F7046FF0DFF5737004306F000000DE
:1049E00093061000E398D7F88327850533E7B700CF
:1049F000232CE5046FF01FF88327850593871700A4
:104A0000232CF5046FF01FF7EF30C0616FF01FF932
:104A10001309440013050900EFB01FDC17C701009C
:104A20001307C7A68327C402032707006376F7008E
:104A300017C70100232CF7A413074001B387E7022F
:104A400017C501001305C5B3930509003305F5002B
:104A5000EFB05FD083278402638607007370043051
:104A60006F00000097C701009387C7A383A70700C3
:104A70000327C40283A7C702E3F2E7F0EFB05FB1F8
:104A80006FF0DFEF130400006FF09FEF630805087D
:104A9000130101FE232C8100232A910023282101E8
:104AA000232631012324410123225101232E110009
:104AB00093090700138A0600930406001389050072
:104AC00013040500EFB01FC1930A050063060A0036
:104AD000832784052320FA000327C40593072000B9
:104AE000232EF4046380F40463FA971093063000D5
:104AF0006388D400930640006396D400630CF70EDD
:104B0000232C2405930710006312F70A83278402DD
:104B100063820702737004306F000000737004300A
:104B20006F0000008327840593871700232CF4046B
:104B30006FF05FFD97C701009387879383A70700F6
:104B40006390070A9304440013850400EFB0DFC8A4
:104B500017C70100130787938327C40203270700A1
:104B60006376F70017C701002322F792130740016D
:104B7000B387E70217C50100130585A093850400DC
:104B80003305F500EFB01FBD97C7010093878791EC
:104B900083A707000327C40283A7C70263F8E700BF
:104BA000638609009307100023A0F9001304100086
:104BB00013850A00EFB09FB1130504008320C101E3
:104BC0000324810183244101032901018329C100B8
:104BD000032A8100832A410013010102678000003B
:104BE0009305840117C50100130585A8EFB09FB692
:104BF0006FF09FF9130400006FF09FFB9307100004
:104C0000E392F4F08327840533E92701232C24055C
:104C10006FF05FEF630A050E130101FE232C810084
:104C2000232A91001304050023282101232E1100BB
:104C30002326310193840500EFB0DFA993072000FC
:104C40008326C405232EF40483278405130710004C
:104C50001309050093871700232CF4046396E608D4
:104C60008327840263860700737004306F0000009E
:104C700097B701009387C77F83A70700639A070848
:104C80009309440013850900EFB01FB517B7010061
:104C90001307C77F8327C402032707006376F70043
:104CA00017B701002324F77E13074001B387E702FB
:104CB00017C501001305C58C938509003305F50060
:104CC000EFB05FA997B701009387C77D83A707005F
:104CD0000327C40283A7C70263F8E70063860400C2
:104CE0009307100023A0F400032481018320C10155
:104CF000832441018329C10013050900032901010F
:104D0000130101026FB09F9C737004306F000000AC
:104D10009305840117C5010013058595EFB09FA386
:104D20006FF05FFA9307050063080506737004309F
:104D300017B701001307477583260700639E060215
:104D400003A6C70593062000130500006316D600CE
:104D500023AE07041305100083270700638C0700A8
:104D600097B701009387077403A707000327470439
:104D7000631C07026780000097B601009386867265
:104D800003A6060083A60600832646049386160023
:104D90002322D6046FF0DFFA97B70100938787705C
:104DA00083A707006FF09FF803A7070083A60700FB
:104DB000832747049387F7FF2322F70483A746043A
:104DC000E39A07FA7360043067800000130101FB67
:104DD0002322910423202105232C4103232A51035C
:104DE000232861032326710323261104232481042D
:104DF000232E310323248103232291032320A103A3
:104E000017B901001309096B17BB0100130BCB691C
:104E100097B401009384846997BA0100938A4A6920
:104E2000130A1000930B90008327090003A70700C3
:104E30006306071683A7C70083A90700EFD09FCF9B
:104E4000EFD0DFD083270B00130C05006368F50C4F
:104E500097B7010023AAA7641306000063763523E1
:104E600003A50400B3858941EFC01FCCEFE00F809C
:104E70006306051603A50400930600001306000050
:104E800093058100EFC08FCAE30005FA83278100F4
:104E9000E3C207FE8329010183A749016386070056
:104EA00013854900EFB05F93EFD05FCA83270B00F3
:104EB000130C05006362F50C8327810017B701000E
:104EC0002324875FE3E8FBFAB317FA0013F70721FF
:104ED0006310072013F7770C6316072A93F707026E
:104EE000E38A07F813850900EF00504F6FF09FF831
:104EF00083A7C70003A4C70083AC0700930944003D
:104F000013850900EFB05F8D832744021305040069
:104F1000E78007008327C4016386470D83270900C4
:104F200003A70700E31607FC03A70A0097B60100D2
:104F300023AC865797B6010023ACF65697B701000D
:104F400023AAE756EFD09FF26FF0DFF283A7C700E6
:104F500003A4C70003AD0700930C440013850C00A5
:104F6000EFB09F878327440213050400E780070002
:104F70008327C401638C470B8327090003A707001D
:104F8000E31607FC03A70A0097B6010023A2F65216
:104F900097B7010023A0E7526FF01FF2EFD09FB93F
:104FA000EFD0DFBA83270B00130C0500E368F5F69A
:104FB00083A70A0003A504009309000003A60700C5
:104FC000B385894117B701002320874F1336160098
:104FD000EFC09FB5EFD09FE9E31E05E8EFB04FDBD0
:104FE0006FF05FE98327840193850900B387FC0094
:104FF00063E2FC0883A7040063860702232A0100FA
:10500000232C9101232E8100EFF08F9D03A5040036
:10501000930600001306000093054101EFB09FB115
:10502000E31E05EE737004306F00000083278401D7
:1050300093850C00B307FD006362FD0883A704009D
:1050400063860702232A0100232CA101232E81005D
:10505000EFF00F9903A5040093060000130600006B
:1050600093054101EFB01FADE31805F073700430F4
:105070006F000000032509002322F4002328840088
:10508000EFB04FF06FF09FE9EFD05FDE83270900AC
:1050900083A7C70003A4C700930C440013850C002A
:1050A000EFB08FF38327C401638A47058327440247
:1050B00013050400E78007006FF0DFDB032509001C
:1050C0002322F40023288400EFB0CFEB6FF0DFEA57
:1050D0008327C10023ACF9006382070AB3878701E5
:1050E00023A2F90023A83901938549006362FC08D3
:1050F00003A50A00EFB00FE96FF0DFD78327840123
:10510000232884003387F9002322E400636AEC0437
:10511000330C3C41636EFC0283A7040063860702E4
:10512000232A0100232C3101232E8100EFF04F8B25
:1051300003A5040093060000130600009305410137
:10514000EFB05F9FE31405F6737004306F0000004A
:1051500003A50A0093850C00EFB0CFE26FF01FF5B6
:105160000325090093850C00EFB0CFE16FF01FF429
:1051700003250900EFB00FE16FF0DFCF737004304B
:105180006F0000008327C10083A6890123A839018D
:105190003387D70023A2E9006362EC06B307FC4023
:1051A00063EAD70683A7490213850900E780070051
:1051B00083A7C901E39047CD83A689018327C10056
:1051C00003A70400B387D70063060702232A010060
:1051D000232CF100232E3101EFF08F8003A5040072
:1051E000930600001306000093054101EFB09F9461
:1051F000E31205C8737004306F0000006374FC0094
:10520000E372F7FA0325090093854900EFB08FD7C1
:105210006FF05FC603A50A0093854900EFB08FD6F3
:105220006FF05FC5130101FF2324810023261100C5
:10523000232291002320210117B401001304042725
:10524000EFF0CF998327040063840704EFF04F9CAD
:1052500083270400638A07029308000013080000F4
:105260009307000013072000930600001306004078
:1052700097B501009385851417050000130545B502
:10528000EFC0DF9E63140506737004306F000000EA
:1052900017B901001309894113050900EFB00FC9BF
:1052A00097B401009384C44113850400EFB00FC884
:1052B000130600009305C0001305400097B70100D6
:1052C00023AA271F97B7010023A4971EEFB08FF2E0
:1052D00017B70100232CA71C6306050297B5010030
:1052E0009385450DEFC00FF16FF05FF68320C1008D
:1052F00003248100832441000329010013010101DB
:1053000067800000737004306F000000638A050A34
:10531000130101FD232A5101930A05001305C00260
:10532000232481022322910223202103232E3101F1
:10533000232C410123261102232861012326710118
:105340001309070093890600130A060093840500D9
:10535000EF00C07013040500630C0502EFF00F8826
:1053600097B701009387871483A70700638E07040C
:10537000EFF00F8A1305440023205401232C9400DE
:10538000232E44012320340323222403EFB00FBC37
:10539000130504008320C1020324810283244102F7
:1053A000032901028329C101032A8101832A4101C2
:1053B000032B0101832BC10013010103678000004F
:1053C000737004306F00000097BB0100938B0B2EAD
:1053D00013850B00EFB08FB517BB0100130B4B2EDD
:1053E00013050B00EFB08FB4130600009305C00047
:1053F0001305400097B7010023AE770B97B7010064
:1054000023A8670BEFB00FDF17B701002320A70A0F
:10541000630A050097B501009385C5F9EFC08FDDDC
:105420006FF01FF5737004306F000000630E050607
:10543000130101FE232C8100232E1100232A910049
:1054400017B4010013048406832804001308050020
:105450001305000063800804930407002322B100B1
:10546000138706002324C100232601019306500060
:1054700063C0B604EFE0DFD693072000630EF504A7
:105480000325040093060000130600009305410065
:10549000EFB04FEA8320C10103248101832441013D
:1054A0001301010267800000737004306F00000078
:1054B00093054100930600001306070013850800BA
:1054C000EFB01FB98320C10103248101832441016E
:1054D0001301010267800000032504009306000009
:1054E0001386040093054100EFB0CFE46FF09FFAFC
:1054F0006306050003250500678000007370043013
:105500006F00000063160500737004306F00000028
:10551000130101FF23261100232481001304050039
:10552000EFE0DFEB032544013334A000EFE05FEE52
:10553000130504008320C10003248100130101012D
:105540006780000063160500737004306F00000070
:10555000130101FF232481001304050023261100F9
:10556000EFE0DFE703240402EFE09FEA8320C100BD
:10557000130504000324810013010101678000006A
:1055800063160500737004306F000000130101FF03
:105590002324810023229100138405009304050035
:1055A00023261100EFE09FE323A08402032481005F
:1055B0008320C10083244100130101016FE05FE5F6
:1055C000130101FF1305C0012324810023261100CC
:1055D000EF00C04813040500630805002320050000
:1055E00013054500EFB08F94130504008320C1001C
:1055F000032481001301010167800000630205029A
:10560000B70700FFB3F7F500638607007370043037
:105610006F000000639A0500737004306F00000093
:10562000737004306F000000130101FE232C810011
:105630002328210123263101232441012322510162
:10564000232E1100232A91009309070013890600D5
:10565000930A060013840500130A0500EFE05FB803
:105660006318050063860900737004306F00000042
:10567000EFD04FCC83240A00B3779400631209045F
:105680006382070463880A009347F4FFB3F7970027
:105690002320FA00EFD08FFD8320C1010324810174
:1056A0001385040003290101832441018329C100DA
:1056B000032A8100832A4100130101026780000050
:1056C000E302F4FCE38809FCB335500193958501AE
:1056D00063060900B7070004B3E5F5001386090067
:1056E000B3E5850013054A00EFE0CFE1EFD00FF8F6
:1056F00063140500EFA0DFE9EFE01FD69317650004
:105700009309050063DA0700B70400019384F4FFEE
:10571000B3F499006FF05FF8EFE05FCC83290A00E3
:10572000B377340163100902638A070063880A00B3
:105730009347F4FFB3F737012320FA00EFE05FCD82
:105740006FF09FFCE31CF4FE6FF05FFE630C05003E
:10575000B70700FFB3F7F500638A070073700430E2
:105760006F000000737004306F000000130101FF30
:105770002324810013040500232611002322910015
:105780002320210113890500EFE05FC58324040075
:105790009345F9FFB3F795002320F400EFE05FC7CE
:1057A0008320C10003248100138504000329010024
:1057B000832441001301010167800000130101FFF0
:1057C000232481001304050023261100EFA09FF07D
:1057D00003240400EFA09FEF8320C1001305040001
:1057E000032481001301010167800000630C0500A0
:1057F000370700FFB3F7E500638A070073700430D2
:105800006F000000737004306F0000006F205004C0
:10581000B70700FFB377F6006386070073700430A4
:105820006F00000063160600737004306F00000004
:10583000130101FE232C810023282101232631019D
:1058400023244101232E1100232A910013890600ED
:1058500093890500130A050013040600EFE05F9822
:10586000631E050463060900737004306F000000B6
:10587000EFD04FAC83240A009385090013050A007A
:10588000B3E49900EFF09FF6B3779400630AF4084D
:1058900083240A00EFD08FDD8320C101032481011E
:1058A0001385040003290101832441018329C100D8
:1058B000032A81001301010267800000EFD08FA747
:1058C00083240A009385090013050A00B3E4340118
:1058D000EFF0DFF1B3F7840063848704E30A09FA89
:1058E000B705000513060900B365B40013054A00A7
:1058F000EFE04FC1EFD08FD763140500EFA05FC971
:10590000EFE09FB5931765009304050063D4070289
:10591000B70700019387F7FFB3F4F4006FF0DFF7E8
:1059200083270A001344F4FFB3F787002320FA000B
:105930006FF05FF6EFE09FAA83240A00B37794002C
:10594000639887009347F4FFB3F797002320FA008A
:10595000EFE01FAC6FF0DFFB130101FF2324810098
:10596000232611001304050023229100EFD08F9C01
:105970008327440063860702032504019304C400BF
:10598000631895006F0080030325040163089502E6
:10599000B7050002EFE04FE183274400E39607FEDE
:1059A00013050400EF008023032481008320C1003D
:1059B00083244100130101016FD04FCB7370043079
:1059C0006F000000630C0500370700FFB3F7E50028
:1059D000638A0700737004306F0000007370043036
:1059E0006F0000006F20C066630C0500B70700FF62
:1059F000B3F7F500638A0700737004306F0000008E
:105A0000737004306F000000130101FF2324810034
:105A1000232291002326110013040500938405001E
:105A2000EFE0DF9B0327040093C7F4FFB377F70091
:105A30002320F400032481008320C100832441003B
:105A4000130101016FE0DF9C63060500032585015A
:105A5000678000001305000067800000130101FF4C
:105A6000232481002326110013040500EFD08F8C1E
:105A700097B70100938747A483A70700639C070497
:105A8000B797010017B70100130707C59387C7FF32
:105A900097B6010023A8E6A217B701002322F7A2B8
:105AA00017B70100232CF7C297B70100938707A10E
:105AB00017B701002322F7C29307100017B70100A0
:105AC000232407A017B70100232A079E17B7010058
:105AD0002324F79E63120402EFD04FB9EF10C05891
:105AE00013040000130504008320C1000324810077
:105AF00013010101678000001305840093773500CE
:105B00006398070CB79701001307F5FF9387A7FF6A
:105B1000E3E4E7FC97B601009386C69A83A70600E4
:105B20006F00400103A70700630A07009386070080
:105B30009307070003A74700E366A7FE17B7010016
:105B40001307C797E38AE7F803A7070013060001C6
:105B50001384870023A0E60003A74700B306A740ED
:105B6000637ED6023388A7002322D80023A2A70091
:105B70008325480097B601009386C6946F00800085
:105B80009306070003A7060003264700E36AB6FE54
:105B90002320E80023A0060103A7470097B70100D0
:105BA0009387079483A70700B387E74017B70100DF
:105BB0002328F792EFD08FABE30204F21305040021
:105BC0008320C100032481001301010167800000CC
:105BD0001375C5FF130545006FF0DFF26308050676
:105BE000130101FF23248100232611001304050063
:105BF000EFC05FF4930584FF0326C4FF17B70100CD
:105C00001307478C6F008000138707008327070066
:105C100083A64700E3EAC6FE232CF4FE2320B70048
:105C200097B701009387C78B03A707008327C4FF9B
:105C3000032481008320C100B387E70017B7010068
:105C40002320F78A130101016FD04FA26780000063
:105C500097B701009387C78803A5070067800000F6
:105C6000678000003367B50013773700930705009E
:105C7000631207049308D6FFB30815011307050044
:105C8000938605006378150303A8060013074700F1
:105C900093864600232E07FFE36817FF9347F5FF1F
:105CA000B387170193F7C7FF93874700B385F500C4
:105CB000B307F5003306C50063F4C70C93864500AF
:105CC00013884700B3B6D70033B8050133E7F500B2
:105CD00093C616001348180013773700B3E6060181
:105CE000133717003377D700330EF640938617002B
:105CF000630807061337AE006314070613532E001C
:105D00001388050093860700130700008328080006
:105D1000130717001308480023A0160193864600B6
:105D2000E36667FE1377CEFFB385E500B387E70030
:105D30006306EE0483C60500138717002380D7008F
:105D4000637EC70283C6150013872700A380D70090
:105D50006376C70203C725002381E7006780000040
:105D6000B307F640B387F5009385150003C7F5FF29
:105D700093861600238FE6FEE398F5FE6780000009
:105D800067800000B367C50093F73700B308C5000C
:105D90006382070E63761511B307A04093F73700AF
:105DA000138737009306500093F5F50F130815007D
:105DB0003383A8401306F6FF6374D700130750001F
:105DC0006368E60E6380070E2300B500130710001A
:105DD000638EE700A300B500130730001308250009
:105DE0006396E700130835002301B500139685007C
:105DF00033E6C500139705013367E6003303F3402C
:105E000093968501B366D70013562300B307F500B8
:105E10001307000023A0D70013071700938747003C
:105E2000E36AC7FE1377C3FFB307E8006300E30824
:105E30002380B70013871700637C1703A380B70084
:105E400013872700637617032381B7001387370072
:105E500063701703A381B70013874700637A1701A4
:105E60002382B7001387570063741701A382B7001A
:105E70006780000093F5F50F13978500B365B700B1
:105E8000139705013367B700E37415FF9307050007
:105E90009387470023AEE7FEE3EC17FF678000001F
:105EA00067800000130805006FF05FF46780000052
:105EB000930705006FF0DFF7834705001307050020
:105EC000638C07001305150083470500E39C07FE5C
:105ED0003305E5406780000013050000678000007F
:105EE000130515008347F5FF9385150003C7F5FFDC
:105EF00063880700E386E7FE3385E740678000009C
:105F0000930700006FF05FFF93070500938515006E
:105F100003C7F5FF93871700A38FE7FEE31807FE7B
:105F20006780000083460500930700026398F6002F
:105F30001305150083460500E38CF6FE938756FD96
:105F400093F7D70F638007049307050093050000BC
:105F5000638806041305000093871700138606FD67
:105F60001317250083C607003305A7001315150076
:105F70003305A600E39206FE638405003305A040C6
:105F800067800000938536FD8346150093B51500A4
:105F900093071500E39006FC130500006FF0DFFD8A
:105FA000130500006780000083A705002380A70079
:105FB00083A705009387170023A0F50067800000E2
:105FC00097A601009386865083A706001737030023
:105FD0001307477313861700B307F7002380A70042
:105FE00097A5010023A4C54E9307A000630AF500FE
:105FF000930700046308F6001305000067800000A3
:10600000E30C06FE370610F0130717008347F7FF6F
:106010002320F6F083A706009387F7FF97A50100DA
:1060200023A6F54AE39207FE1305000067800000EF
:10603000130101EB2322911423202115232A51134C
:10604000232481132326111423248114232E311396
:10605000232C411323286113232671132322911328
:106060002320A113232EB1119304050013890500E9
:106070002326C100130C5002930A900083470900A5
:1060800063888703638C070603A404006F00800005
:10609000638607062300F40003A404001309190013
:1060A0001304140023A0840083470900E39287FFB0
:1060B000034619009308190093860800130D000287
:1060C0009309F0FF130AF0FF1308000013055005B1
:1060D0009307D6FD93F7F70F13891600636EF53A11
:1060E00017A70100130707F293972700B387E7006C
:1060F00083A70700B387E700678007008320C114E8
:106100000324811483244114032901148329C11316
:10611000032A8113832A4113032B0113832BC112FA
:10612000032C8112832C4112032D0112832DC111E6
:106130001301011567800000930C800023240100E7
:106140009307100063DA071D8327C10003A404002E
:10615000938B770093F68BFF03AB060083A9460071
:10616000938786002326F10013860C009306000017
:1061700013050B0093850900EF1050212328A1007F
:106180009307000063803733930D4101930B100098
:1061900013860C009306000013050B00938509007D
:1061A000EF10805B9306000013860C00130B0500B4
:1061B00093890500EF10901D8327810023A0AD0077
:1061C00093861B00938D4D0063863701938B0600E9
:1061D0006FF01FFCE37C9BFF63D246039307040030
:1061E0002380A70103A40400130AFAFF93071400F5
:1061F00023A0F40013840700E3C446FF93962B000A
:1062000093070101B386D7006F008002938777055B
:106210002300F40003A40400938BFBFF93871B006F
:106220001304140023A084009386C6FFE358F0E40F
:1062300083A70600E3ECFAFC938707036FF05FFD8A
:1062400083A70400930600030327C1002380D7001F
:1062500083A7040093064700930C000113861700E0
:1062600023A0C40013068007A380C70003A4040072
:1062700023240100930707001304140023A08400C3
:1062800003AB0700930900002326D1006FF0DFED78
:106290008327C10083AC0700938B470063880C28D9
:1062A000635C40259307D002631EFD2083C70C006A
:1062B0006388070263D8092483A60400938C1C001A
:1062C000130AFAFF2380F60003A404001304140049
:1062D00023A0840083C70C00E39E07FC63524003A5
:1062E00003A40400930700022300F40003A40400A5
:1062F000130AFAFF1304140023A08400E3160AFE15
:10630000232671016FF09FD723240100930710000B
:10631000930CA000E3CA07E38327C10003A4040091
:10632000938647006FF0DFF503C616009306090059
:106330006FF01FDA83A70400930650022380D70072
:1063400003A404001304140023A084006FF01FD3DF
:10635000930C0001232401006FF09FDE8327C1000E
:1063600003C616009306090083A907009387470018
:106370002326F100E35E0AD4138A09009309F0FF93
:106380006FF01FD503C61600130DD0029306090047
:106390006FF01FD49347FAFF93D7F74103C6160057
:1063A000337AFA00930609006FF09FD203C61600F5
:1063B000130D0003930609006FF09FD183C51600EB
:1063C000930906FD93060900938705FD13860500D2
:1063D000E3E2FAFA93972900B3893701938616000E
:1063E00093991900B389B90083C50600938909FD03
:1063F000938705FD13860500E3FEFAFC6FF09FF717
:106400000327C10083A70400832607001307470062
:106410002326E1002380D70003A404001304140002
:1064200023A084006FF09FC59307100063D4070F6B
:106430008327C1009386770093F686FF93878600B3
:106440002326F10083A9460083A7060063DE090E18
:1064500083A604001306D002B307F0402380C600D1
:1064600003A40400B336F000B30930411304140050
:1064700023A08400138B0700B389D940930CA0009C
:10648000232401006FF05FCE03C616001308180026
:10649000930609006FF0DFC383A704001389080087
:1064A0006FF09FE9E3729BCF93071000930B0000FE
:1064B00093061000E3C447D36FF05FD497AC01009C
:1064C000938C4CF09385090013850C00EF0010614C
:1064D000330AAA406352400303A404002300A4012A
:1064E00003A40400130AFAFF1304140023A0840079
:1064F000E3160AFE130A000083C70C00E38207E0DC
:10650000E3CC09DA9389F9FF1307F0FFE396E9DAA0
:106510006FF0DFDC8327C1009386470083A7070065
:106520002326D10093D9F7416FF05FF26356400103
:106530009307D002E314FDF897AC0100938C8CE82C
:10654000930780026FF01FD7138B0700930CA000F6
:106550002324010003A404006FF01FC1130101EB09
:10656000232E3113B70900409387F9FF23248114A8
:1065700023229114232C4113232A5113232611146F
:10658000232021152328611323267113232481132B
:10659000232291132320A113232EB111130A0500E6
:1065A0002324B10017A40100130444F2973A030016
:1065B000938A4A1597A40100938444BA2326F100D4
:1065C000930550021305A00013080004B70610F04D
:1065D00083470A00638EB7046388070A0327040011
:1065E000130A1A00130617003387EA0097A8010060
:1065F00023AEC8EC2300F7006380A708E31A06FD6A
:106600001737030013070710130717008347F7FF17
:1066100023A0F6F0832704009387F7FF17A6010055
:106620002326F6EAE39207FE83470A00E396B7FAC9
:1066300083461A0013051A0013070500930B000286
:10664000130BF0FF130CF0FF130800009305500527
:10665000930890009387D6FD93F7F70F130A17005E
:1066600063ECF54493972700B387970083A707004F
:10667000B387970067800700173703001307870861
:10668000E31406F86FF0DFF48320C11403248114AF
:1066900083244114032901148329C113032A81137C
:1066A000832A4113032B0113832BC112032C811264
:1066B000832C4112032D0112832DC11113010115E9
:1066C00067800000930C8000130D000093071000FA
:1066D00063DA0721832781009387770093F787FF89
:1066E00083AD070003AB4700138787002324E10035
:1066F00013860C009306000013850D0093050B0014
:10670000EF10C0482328A10063086D45130941011B
:106710009309100013860C009306000013850D00EA
:1067200093050B00EF10400313860C009306000046
:10673000930D0500138B0500EF1040452320A900A1
:106740009389190013094900E3166DFDE3F49DFDDB
:1067500013060004B70610F063D4890383270400EE
:1067600013871700B387FA0097A5010023A0E5D689
:1067700023807701630AC706130CFCFFE3C089FF7F
:106780008327C1001305C10093089000B386F90068
:106790009396260093070101B386D7001308A00043
:1067A00013030004370610F0E38CA6E083A706006D
:1067B0009305000363F4F8009305700503270400B4
:1067C000B387B700930517003387EA0017AE0100BF
:1067D000232EBECE2300F70063860737638C653215
:1067E0009386C6FF6FF05FFC17370300130787F12E
:1067F000130717008347F7FF23A0F6F08327040051
:106800009387F7FF97A5010023A2F5CCE39207FE3B
:10681000130CFCFF6FF09FF683270400130600049F
:106820001387170097A5010023A2E5CAB386FA00D3
:10683000930500032380B6006308C75093872700A1
:1068400097A6010023A4F6C83387EA0093068007C1
:106850002300D700173703001307C7EAB70610F065
:106860006392C702130717008347F7FF23A0F6F0D0
:10687000832704009387F7FF17A601002328F6C497
:10688000E39207FE83278100930C0001130D0000A3
:106890009387470003278100130B0000832D070017
:1068A0002324F1006FF0DFE48327810083AC07002D
:1068B00013894700638E0C4C6358802B9307D002DA
:1068C0006394FB3E03C70C00930507006314072A7B
:1068D0006F00002F93071000930CA000130D000011
:1068E000E3CA07DF83278100938747006FF09FFA91
:1068F000832781008346170013070A0003AB0700B4
:10690000938747002324F100E3560CD4130C0B00AB
:10691000130BF0FF6FF01FD483461700930BD002C8
:1069200013070A006FF01FD39347FCFF93D7F7417B
:1069300083461700337CFC0013070A006FF09FD1D9
:1069400083461700930B000313070A006FF09FD0D4
:1069500003461700138B06FD13070A00930706FD75
:1069600093060600E3E2F8FA93172B00B38767015A
:106970001307170093971700B387C7000346070054
:10698000138B07FD930706FD93060600E3FEF8FC54
:106990006FF09FF783258100832704001306A00072
:1069A00003A7050093861700B387FA0017A5010017
:1069B000232ED5B02380E700138945006300C73636
:1069C000930700046384F62A232421016FF05FBF3C
:1069D0009307100063DE0735832781001387770054
:1069E000137787FF930787002324F100032B4700C9
:1069F0008327070063560B3E032704001306000499
:106A00009306170097A5010023A2D5AC3387EA00AF
:106A10009305D0022300B700638CC638B307F0405B
:106A20003337F000330B6041938D0700330BEB409D
:106A3000930CA000130D00006FF09FCB834617004E
:106A40001308180013070A006FF0DFC08346170011
:106A500013070A006FF01FC0832704009306000489
:106A60001387170017A601002322E6A6B387FA00B2
:106A7000130650022380C700E314D7B4173703006E
:106A8000130747C8B70610F0130717008347F7FF2F
:106A900023A0F6F0832704009387F7FF17A60100D1
:106AA0002326F6A2E39207FE6FF09FB1930C00013C
:106AB000130D00006FF09FC18327040093060004AC
:106AC000130A05001387170017A601002320E6A06C
:106AD000B387FA00130650022380C700E312D7AE33
:106AE00017370300130707C2B70610F01307170084
:106AF0008347F7FF23A0F6F0832704009387F7FF6F
:106B000017A601002324F69CE39207FE130A050052
:106B10006FF01FAB173703001307C7BE130717002B
:106B20008347F7FF2320F6F0832704009387F7FFBE
:106B300097A5010023ACF598E39207FE9386C6FF64
:106B40006FF09FC6173703001307C7BBE39805FC18
:106B50009386C6FF6FF05FC5E3FA9DBB93091000F3
:106B60006FF01FBF130C000003C70C009305070054
:106B7000E30C07E49308F0FF1305A00013080004DA
:106B8000B70610F0635E0B0C832704001386170012
:106B9000B387FA0017A30100232AC3922380E700DA
:106BA0006382A5086308060B938C1C0003C70C00C6
:106BB000130CFCFF93050700E31607FCE35680E186
:106BC000832704009305000213060004B70610F0A3
:106BD0006F00C000130CFCFFE3080CDE13871700E6
:106BE000B387FA002380B70017A501002320E58EA4
:106BF00093070700E310C7FE17370300130787B09A
:106C0000130717008347F7FF23A0F6F0832704003C
:106C10009387F7FF17A50100232AF58AE39207FE61
:106C20006FF05FFB173703001307C7ADE30E06F6DF
:106C3000130717008347F7FF23A0F6F0832704000C
:106C40009387F7FF17A601002322F688E39207FE39
:106C50006FF09FF5173703001307C7AA6FF05FFDAA
:106C6000130BFBFFE3121BF36FF05FF51737030005
:106C7000130747A9B70610F0130717008347F7FF5C
:106C800023A0F6F0832704009387F7FF17A60100DF
:106C9000232EF682E39207FE232421016FF05F92F8
:106CA000979C0100938C0C7293050B0013850C00CC
:106CB000EF00C062330CAC40E35880EB8327040044
:106CC00013060004B70610F06F00C000130CFCFFA1
:106CD000E30A0CE813871700B387FA0023807701D3
:106CE0009795010023A4E57E93070700E310C7FEF4
:106CF00017370300130707A1130717008347F7FF90
:106D000023A0F6F0832704009387F7FF97950100EF
:106D100023AEF57AE39207FE6FF05FFB17370300AF
:106D20001307479EE39806F4232421016FF05F893F
:106D3000832781001387470083A707002324E100EE
:106D400013DBF7416FF01FCB173703001307879B47
:106D5000B70610F0130717008347F7FF23A0F6F0DC
:106D6000832704009387F7FF179601002320F67608
:106D7000E39207FE93071000179701002328F7748A
:106D80009307800717370300230EF7966FF09FAF26
:106D9000635680019307D002E394FBF0979C0100B7
:106DA000938C4C6213078002930580026FF09FDC86
:106DB0009736030093860695370610F093861600E3
:106DC00003C7F6FF2320E6F0032704001307F7FFAD
:106DD0009795010023ACE56EE31207FE6FF01FC428
:106DE000938D0700930CA000130D00006FF05F90CF
:106DF000B70710F023A0A7F26F000000130101FCF9
:106E0000130341022322B10293050300232E110034
:106E10002324C1022326D1022328E102232AF102DE
:106E2000232C0103232E110323266100EFF00FF31F
:106E30008320C101130500001301010467800000D5
:106E4000130101FB13038103232481022326A100E4
:106E5000232CC10213040500130603001305C1000F
:106E6000232611022322F104232ED1022320E10440
:106E70002324010523261105232E6100EFF04F9BEB
:106E80008327C100238007000325C1008320C1029E
:106E9000330585400324810213010105678000004A
:106EA000B70710F083A647F403A607F403A747F437
:106EB000E31AD7FEB7160000938606FAB306D6008B
:106EC00033B6C600B305E60023A4D7F423A6B7F46F
:106ED00067800000B70710F003A747F403A607F484
:106EE00083A647F4E31AD7FEB7160000938606FA86
:106EF000B306D60033B6C60023A4D7F4B305E60024
:106F000023A6B7F49307000873A0473067800000FA
:106F1000130101FF2324810023261100979701000C
:106F20009387475B179401001304845A03A7070053
:106F3000832704001306F07C9306470693874706D1
:106F40009795010023A8D5589795010023A2F558DD
:106F5000634AD6008320C10003248100130101018C
:106F600067800000130747899797010023A4E7561D
:106F7000EF00C02D930710006316F50203270400ED
:106F8000B71700009387F77613050000E3D4E7FCFA
:106F9000EFF01FE6032481008320C10013010101EB
:106FA0006FB05FB81795010013054542EFF01FE57C
:106FB00013052000EFF0DFE3032481008320C100EC
:106FC000130101016FB01FB617950100130585412C
:106FD0006FF0DFE217950100130545416FF01FE2E6
:106FE000130101FF23248100232291002326110095
:106FF000B7140000179401001304C43F938784382A
:10700000130000009387F7FFE39C07FE13050400BD
:10701000EFF0DFDE6FF09FFE130500006F00C01A77
:10702000130101FF23261100EF0040221307100077
:1070300093070000631AE5008320C1001385070051
:107040001301010167800000179501001305053841
:10705000EFF0DFDA8320C1009307200013850700DB
:107060001301010167800000737004306F0000009D
:1070700067800000737004306F000000130101FE90
:10708000232C8100232A910023263101232441014E
:1070900023225101232E1100232821010329050059
:1070A000979A0100938A8A43EFE05FB39724030025
:1070B0009384446D179A0100130A0A3517040000DF
:1070C0001304C40797990100938989341305803EFE
:1070D000EFC00F8593080000130800009387040099
:1070E00013070900930600001306004093050A00E9
:1070F000130504001723030023260368EFA01FB71E
:10710000930700001307090093080000130800000C
:1071100093860400130600409385090013050400BC
:10712000EFA0DFB483D70A009387170017970100F9
:107130002316F73A6FF09FF9130101FE232E110079
:10714000232C8100232A910023282101630A0500B2
:10715000032405001309200093049005631804021A
:10716000930420001304900523249100232681001A
:10717000832781000327C1001305800CB387E70232
:107180002326F100EFB0DFF96FF01FFE2324210169
:1071900023269100032781008327C1001305800C5B
:1071A000B387E7022326F100EFB09FF71305000035
:1071B000EFB01FF713050400EFA0DFEB130500008D
:1071C000EFA05FEB6FF09FF9130101FF2324810013
:1071D000130405001305400023261100EFE01F886B
:1071E0009307000013070400930605002320850081
:1071F00093080000130800001306C0439795010090
:107200009385852117050000130585E7EFA01FA6CC
:10721000EFB05F9F9797010023A0A72C97970100DD
:107220009387872B03A707001307170023A0E70006
:1072300003A707001307170023A0E7008320C1005E
:10724000032481001301010167800000130101FF85
:1072500023248100232611009797010083D7072854
:10726000179701000357472813040000630EF70027
:10727000979701009387872683D707001304100090
:10728000179701002312F726EFB0DF9797970100B9
:107290009387872403A707006366E50283A7070097
:1072A0008320C1003305F540133545003305A04068
:1072B0003374A400130504000324810013010101A9
:1072C0006780000013040000130504008320C10040
:1072D000032481001301010167800000B305B5009C
:1072E000930705006386B70003C70700631607000E
:1072F0003385A74067800000938717006FF09FFEDB
:107300009308000063DC05003305A040B337A000FC
:10731000B305B040B385F5409308F0FF63DA06008B
:107320003306C040B337C000B306D040B386F64042
:107330001308060013830600930705001387050052
:1073400063980624979601009386C6F663F8C50EE7
:10735000370E0100637AC60D130EF00F6374CE0072
:1073600013038000335E6600B386C60103CE0600B9
:10737000330E6E00130300023303C341630C03009A
:10738000B3956500335EC501331866003367BE00F0
:10739000B3176500135E0801B355C7031315080141
:1073A0001355050193D607013376C703B305B5021C
:1073B00013160601B366D60063FAB600B38606015B
:1073C00063E6060163F4B600B3860601B386B640F1
:1073D00033F7C6039397070193D70701B3D6C603C4
:1073E000B306D50213150701B367F50063FAD7009A
:1073F000B387070163E6070163F4D700B38707018A
:10740000B387D74033D5670093050000638C08002D
:10741000B307A0403337F000B305B0401385070031
:10742000B385E54067800000370E000113030001BB
:10743000E36AC6F3130380016FF0DFF26316060000
:107440001308100033586802370701006372E80A16
:107450001307F00F637407011303800033576800AC
:10746000B386E60003C60600330666001303000277
:107470003303C34063180308B385054193560801DD
:10748000131508011355050113D6070133F7D5026B
:10749000B3D5D502131707013367C700B305B5028B
:1074A000637AB70033070701636607016374B700A7
:1074B00033070701B305B74033F7D50293970701A8
:1074C00093D70701B3D5D502B305B502131507014C
:1074D000B367F50063FAB700B387070163E60701F6
:1074E00063F4B700B3870701B387B7406FF09FF12C
:1074F0003707000113030001E362E8F6130380017C
:107500006FF0DFF53318680033DEC500935E0801C5
:107510003356C500B31765003355DE03B3956500D8
:107520003366B6009315080193D5050193560601FD
:107530003377DE033385A502131707013367D700BE
:10754000637AA70033070701636607016374A70026
:1075500033070701B306A74033F7D6031316060116
:1075600013560601B3D6D60313170701B386D50207
:10757000B365C70063FAD500B385050163E605016D
:1075800063F4D500B3850501B385D5406FF01FEFD7
:10759000E3EED5E63708010063FC0605930EF00F15
:1075A00033B8DE001318380033DE060117930100EC
:1075B000130343D03303C301834E0300130E0002B1
:1075C000B38E0E01330EDE41631E0E0263E4B6007D
:1075D000636AC500B307C540B385D5403335F500B0
:1075E0003387A54013850700930507006FF01FE25E
:1075F0003703000113080001E3E866FA130880016D
:107600006FF09FFA3357D601B396C601B366D70021
:10761000B357D50133D7D501B395C501B3E7B7004B
:1076200093D506013373B702139F0601135F0F0151
:1076300013D807013316C6013315C5013357B702F6
:107640001313030133680301B30FEF0213030700A1
:10765000637EF8013308D8001303F7FF6368D8008E
:107660006376F8011303E7FF3308D8003308F841C5
:10767000B37FB8023358B802939F0F01B3050F03CD
:10768000139F0701135F0F0133EFEF01130708008A
:10769000637EBF00330FDF001307F8FF6368DF006E
:1076A0006376BF001307E8FF330FDF0013130301F6
:1076B000B70F01003363E3009387FFFF1358060100
:1076C000330FBF40B375F30013530301B377F600D4
:1076D0003387F502B307F302B385050333030303CE
:1076E000B385F500135807013308B8006374F80038
:1076F0003303F301B70701009387F7FF93550801A0
:107700003378F800131808013377F700B385650064
:107710003307E8006366BF00631EBF00637CE500BB
:107720003306C7403337C700B385D540B385E5403E
:10773000130706003307E5403335E500B305BF40C6
:10774000B385A540B397D5013357C70133E5E700AB
:10775000B3D5C5016FF09FCB9387050013080600D2
:107760001387060013030500639606289798010007
:10777000938848B463F6C50E370701006378E60CBA
:107780001307F00F3337C70013173700B356E6005F
:10779000B388D80083C608003387E600930600024A
:1077A000B386E640638C0600B397D7003357E500F5
:1077B0003318D600B365F7003313D500135508010D
:1077C000B3D7A502131608011356060193560301F9
:1077D00033F7A502B305F60213170701B366D70006
:1077E0001387070063FEB600B38606011387F7FF11
:1077F00063E8060163F6B6001387E7FFB386060168
:10780000B386B640B3F7A602131303011353030163
:10781000B3D6A6029397070133E36700B305D602F8
:1078200013850600637CB300330368001385F6FFFD
:10783000636603016374B3001385E6FF1317070142
:107840003367A700930500006F00400EB7060001E4
:1078500013070001E36CD6F2130780016FF01FF3EA
:10786000631606009306100033D8C602B70601005F
:107870006372D80C9306F00F63F4060113078000BF
:10788000B356E800B388D80083C60800B386E60084
:10789000130700023307D7406318070AB38707416D
:1078A00093051000135608019318080193D8080196
:1078B0009356030133F7C702B3D7C7021317070163
:1078C000B366D7003385F8021387070063FEA6006E
:1078D000B38606011387F7FF63E8060163F6A60087
:1078E0001387E7FFB3860601B386A640B3F7C60247
:1078F0001313030113530301B3D6C6029397070171
:1079000033E36700B388D80213850600637C130154
:10791000330368001385F6FF636603016374130184
:107920001385E6FF131707013367A7001305070048
:1079300067800000B706000113070001E362D8F476
:10794000130780016FF0DFF33318E800B3D5D700D9
:107950003313E500B356D50013550801B397E7007C
:1079600033F7A502B3E8F6009317080193D7070190
:1079700013D60801B3D5A502131707013367C70053
:10798000B386B70213860500637ED700330707016D
:107990001386F5FF636807016376D7001386E5FF5A
:1079A00033070701B306D74033F7A60293980801BF
:1079B00093D80801B3D6A60213170701B385D702DF
:1079C000B36717011387060063FEB700B38707018B
:1079D0001387F6FF63E8070163F6B7001387E6FF36
:1079E000B3870701B387B74093150601B3E5E500F8
:1079F0006FF05FEB63E6D5183707010063F4E60428
:107A00001308F00F3337D8001317370033D8E600C8
:107A1000979501009385058AB385050103C8050084
:107A2000930500023308E800B3850541639605021B
:107A300013071000E3ECF6EE3335C50013471500CD
:107A40006FF0DFEEB705000113070001E3E0B6FCBD
:107A5000130780016FF09FFB33570601B396B60002
:107A6000B366D70093DE060133D70701B378D70397
:107A7000B397B700335805013363F80093970601B5
:107A800093D70701135803013316B6003357D703B2
:107A90009398080133E80801338FE702130E0700BB
:107AA000637EE8013308D800130EF7FF6368D8003F
:107AB0006376E801130EE7FF3308D8003308E84186
:107AC000B378D8033358D80393980801B38E0703CB
:107AD0009317030193D70701B3E7F80013070800D2
:107AE00063FED701B387D7001307F8FF63E8D70019
:107AF00063F6D7011307E8FFB387D700131E0E0103
:107B0000B387D741B70E01003367EE001388FEFF3D
:107B100033730701935807013378060113560601A2
:107B2000330E03033388080393560E013303C30255
:107B300033030301B3866600B388C80263F4060109
:107B4000B388D80113D60601B308160163E61703FC
:107B5000E39A17CFB70701009387F7FFB3F6F60054
:107B600093960601337EFE003315B500B386C60139
:107B700093050000E37CD5DA1307F7FF6FF09FCC85
:107B800093050000130700006FF05FDA930806000A
:107B9000138706009307050013880500639C0622DF
:107BA000978601009386067163FCC50C37030100BC
:107BB000637E660A1303F00F6374C300130780002B
:107BC0003353E600B386660003CE060013030002BB
:107BD000330EEE003303C341630C0300B39565001D
:107BE000335EC501B31866003368BE00B317650085
:107BF00013D608013377C802139508011355050100
:107C000093D607013358C80213170701B366D7008C
:107C10003308050363FA0601B386160163E616010D
:107C200063F40601B3861601B386064133F7C60234
:107C30009397070193D70701B3D6C602B306D502BF
:107C400013150701B367F50063FAD700B38717016F
:107C500063E6170163F4D700B3871701B387D740F2
:107C600033D56700930500006780000037030001EB
:107C700013070001E36666F4130780016FF05FF4F9
:107C80006316060013061000B358160337060100EA
:107C900063F2C80A1306F00F63741601130780001D
:107CA00033D6E800B386C60003CE060013030002F5
:107CB000330EEE003303C34163180308B385154147
:107CC00013D70801139508011355050113D60701B1
:107CD000B3F6E502B3D5E50293960601B3E6C60016
:107CE000B305B50263FAB600B386160163E6160162
:107CF00063F4B600B3861601B385B640B3F6E50269
:107D00009397070193D70701B3D5E502B305B502F1
:107D100013950601B367F50063FAB700B38717013F
:107D200063E6170163F4B700B3871701B387B74061
:107D30006FF01FF33706000113070001E3E2C8F6F6
:107D4000130780016FF0DFF5B398680033D7C501E2
:107D5000B3176500335EC50113D50801B376A702DA
:107D6000B3956500336EBE009395080193D5050168
:107D700013560E013357A70293960601B3E6C600C9
:107D80003387E50263FAE600B386160163E616015F
:107D900063F4E600B38616013386E640B376A602A6
:107DA000131E0E01135E0E013356A60293960601B2
:107DB0003386C502B3E5C60163FAC500B385150174
:107DC00063E6150163F4C500B3851501B385C540AD
:107DD0006FF01FEFE3EAD5E83707010063FCE60424
:107DE000930EF00F33B7DE001317370033D3E600DE
:107DF000978801009388084CB388680083CE0800F8
:107E0000130E0002B38EEE00330EDE41631E0E022F
:107E100063E4B600636AC500B307C540B385D540C7
:107E20003335F5003388A540138507009305080016
:107E30006FF09FE3B708000113070001E3E816FBAA
:107E4000130780016FF09FFA3357D601B396C6012E
:107E5000B366D700B357D50133D7D501B395C50164
:107E6000B3E7B70093D506013373B702139F06013A
:107E7000135F0F0193D807013316C6013315C501EF
:107E80003357B70213130301B36813013308EF022A
:107E90001303070063FE0801B388D8001303F7FF3C
:107EA00063E8D80063F608011303E7FFB388D8003E
:107EB000B3880841B3FFB802B3D8B802939F0F014B
:107EC000B3051F03139F0701135F0F0133EFEF018A
:107ED00013870800637EBF00330FDF001387F8FFAE
:107EE0006368DF006376BF001387E8FF330FDF00AE
:107EF00013130301B70801003363E3009387F8FF0E
:107F000013580601330FBF40B375F3001353030139
:107F1000B377F6003387F502B307F302B3850503A1
:107F200033030303B385F500135807013308B80082
:107F30006374F80033031301B70701009387F7FF59
:107F4000935508013378F800131808013377F700C8
:107F5000B38565003307E8006366BF00631EBF009A
:107F6000637CE5003306C7403337C700B385D5408F
:107F7000B385E540130706003307E5403335E500D8
:107F8000B305BF40B385A540B397D5013357C701AB
:107F900033E5E700B3D5C5016FF01FCD978701002A
:107FA0009387475083A60700178701001307474EA2
:107FB0000327070023A2A600637EE50017870100C0
:107FC0001307C74D0325070083A5070093854500C8
:107FD0006F804FFB130101FF232481002326110032
:107FE000178701001307C74B13040500032507007B
:107FF00083A5070093854500EF80CFF897870100A0
:108000009387474783A707006376F40097870100AB
:1080100023A287468320C1000324810013010101AC
:1080200067800000978701009387C74703A7070071
:1080300083A60700832747049387F7FF2322F704CB
:1080400083A74604639407007360043067800000D0
:10805000130101FE232C8100232A91001304050043
:108060009384050023282101232631012324410183
:1080700023225101232E1100EFA0DFAB8327040040
:1080800003290401B7090001B3E59700930AC4006E
:108090002320B400930400009389F9FF370A0002FB
:1080A0000327040063822A0503260900130509003B
:1080B000B3654701B37636019317560033F7E600F0
:1080C0000329490063C60700631607006FF05FFDD0
:1080D000E398E6FC9317760063D40700B3E4D4007A
:1080E000EFB09FEC6FF0DFFB93C4F4FFB3F4E40058
:1080F00023209400EFA09FD7032504008320C10113
:108100000324810183244101032901018329C10042
:10811000032A8100832A41001301010267800000C5
:10812000130101FF13050000232611002324810001
:10813000EFF08F8917F7FFFF1307C7DD93060000E5
:108140001306100093054006178501001305052B43
:10815000EFD0CF9B6302050213040500EFA01F9F21
:108160001306050013070000930600009305100096
:1081700013050400EFD08FABEFA00FE98320C100FF
:108180000324810013050000130101016780000032
:02000004800278
:100000002863FEFF9864FEFF3463FEFF9864FEFFE2
:100010009864FEFF9864FEFF9864FEFF5C63FEFF39
:100020009864FEFF9864FEFF8463FEFF9463FEFF06
:100030009864FEFFAC63FEFFBC63FEFFBC63FEFF83
:10004000BC63FEFFBC63FEFFBC63FEFFBC63FEFF40
:10005000BC63FEFFBC63FEFFBC63FEFF9864FEFF53
:100060009864FEFF9864FEFF9864FEFF9864FEFFAC
:100070009864FEFF9864FEFF9864FEFF9864FEFF9C
:100080009864FEFF9864FEFF9864FEFF9864FEFF8C
:100090009864FEFF9864FEFF9864FEFF9864FEFF7C
:1000A0009864FEFF9864FEFF9864FEFF9864FEFF6C
:1000B0009864FEFF9864FEFF9864FEFF9864FEFF5C
:1000C0009864FEFF9864FEFF9864FEFF9864FEFF4C
:1000D0009864FEFF9864FEFF9864FEFF9864FEFF3C
:1000E0009864FEFF9864FEFF9864FEFF9864FEFF2C
:1000F0009864FEFF9864FEFF9864FEFF9864FEFF1C
:100100000064FEFF2864FEFF9864FEFF9864FEFF13
:100110009864FEFF9864FEFF9864FEFF9864FEFFFB
:100120009864FEFF8864FEFF9864FEFF9864FEFFFB
:100130003861FEFF4062FEFF9864FEFF9864FEFF98
:100140009062FEFF9864FEFF0863FEFF9864FEFF66
:100150009864FEFF5063FEFFF468FEFF6069FEFFD7
:100160000069FEFF6069FEFF6069FEFF6069FEFFD7
:100170006069FEFF9867FEFF6069FEFF6069FEFF31
:10018000C067FEFFD067FEFF6069FEFFE867FEFF05
:10019000F867FEFFF867FEFFF867FEFFF867FEFFEF
:1001A000F867FEFFF867FEFFF867FEFFF867FEFFDF
:1001B000F867FEFF6069FEFF6069FEFF6069FEFF91
:1001C0006069FEFF6069FEFF6069FEFF6069FEFF17
:1001D0006069FEFF6069FEFF6069FEFF6069FEFF07
:1001E0006069FEFF6069FEFF6069FEFF6069FEFFF7
:1001F0006069FEFF6069FEFF6069FEFF6069FEFFE7
:100200006069FEFF6069FEFF6069FEFF6069FEFFD6
:100210006069FEFF6069FEFF6069FEFF6069FEFFC6
:100220006069FEFF6069FEFF6069FEFF6069FEFFB6
:100230006069FEFF6069FEFF6069FEFF6069FEFFA6
:100240006069FEFF6069FEFF6069FEFF6069FEFF96
:100250006069FEFF6069FEFF3C68FEFF7868FEFF94
:100260006069FEFF6069FEFF6069FEFF6069FEFF76
:100270006069FEFF6069FEFF6069FEFFE468FEFFE3
:100280006069FEFF6069FEFF6C65FEFFC066FEFFF1
:100290006069FEFF6069FEFF5067FEFF6069FEFF58
:1002A0007C67FEFF6069FEFF6069FEFF5469FEFF28
:1002B000000102020303030304040404040404040D
:1002C00005050505050505050505050505050505DE
:1002D00006060606060606060606060606060606BE
:1002E00006060606060606060606060606060606AE
:1002F000070707070707070707070707070707078E
:10030000070707070707070707070707070707077D
:10031000070707070707070707070707070707076D
:10032000070707070707070707070707070707075D
:10033000080808080808080808080808080808083D
:10034000080808080808080808080808080808082D
:10035000080808080808080808080808080808081D
:10036000080808080808080808080808080808080D
:1003700008080808080808080808080808080808FD
:1003800008080808080808080808080808080808ED
:1003900008080808080808080808080808080808DD
:1003A00008080808080808080808080808080808CD
:1003B000546D725100000000546D7220537663003A
:1003C000286E756C6C2900004572726F7220696E20
:1003D000206465617468207461736B73200D0A007A
:1003E0006D69616F750A00006D69616F75320A0091
:1003F00068756E6772790A00436865636B54696D4E
:1004000065720000535549434944310053554943EF
:0C0410004944320043524541544F520011
:10041C001000000000000000017A5200017C010174
:10042C001B0D02001000000018000000C86EFEFF3B
:10043C005804000000000000100000002C00000018
:10044C000C73FEFF340400000000000010000000DC
:10045C00400000002C77FEFF10040000000000009C
:0A04DC00FC8F010009000000FF0F73
:0204E600000014
:040000058000004037
:00000001FF
